:1080000000000120B911010029E4000029E400006A
:1080100029E4000029E4000029E400000000000039
:1080200000000000000000000000000029E4000043
:1080300029E400000000000029E40000AD850000F4
:1080400029E4000029E4000029E4000029E40000FC
:1080500029E4000029E4000029E4000029E40000EC
:1080600029E4000029E4000029E4000029E40000DC
:1080700029E4000029E4000029E4000029E40000CC
:1080800029E4000029E4000029E4000029E40000BC
:1080900029E4000029E4000029E4000029E40000AC
:1080A00029E400001DD3000029E4000029E40000B9
:1080B00029E4000029E4000029E4000029E400008C
:1080C00029E4000029E4000029E4000029E400007C
:1080D00029E4000029E4000029E40000EDCE0000BE
:1080E00029E4000029E4000029E4000029E400005C
:1080F00029E4000029E4000029E4000029E400004C
:1081000029E4000029E4000029E4000029E400003B
:1081100029E40000D1F6000029E4000029E4000071
:1081200029E4000029E4000029E4000029E400001B
:1081300029E4000029E4000029E4000029E400000B
:1081400029E4000029E400001187000029E4000070
:1081500029E4000029E4000029E4000029E40000EB
:1081600029E4000039CF000029E4000029E40000E0
:1081700029E4000029E4000029E4000029E40000CB
:0881800029E4000029E40000DD
:10840000FFFFFFFFFFFFFFFFFFFFFFFF7EF9FFFF03
:1084100010B5054C237833B9044B13B10448AFF3BE
:1084200000800123237010BD0086FF1F00000000A4
:108430007419010008B5064B1BB106480649AFF395
:1084400000800648036813B1054B03B1984708BD87
:1084500000000000741901000486FF1F6885FF1FDB
:108460000000000080F31188704741F238022C4B65
:10847000995841F4785199502A4A927902F00C02A5
:108480000C2A4CD041F244022749995003F5583345
:108490009A78120703D59A7842F008029A70204B16
:1084A000224941F24402995041F204015A5842F4DF
:1084B000803242F0C0025A501A6842F440221A60D8
:1084C00003F5E83324225A70194A80211170A22240
:1084D0001A70DA7802F01F02DA7003221A71002291
:1084E0005A719A799007FCD59A79D106FCD40D4B34
:1084F0009A7902F00C02082AF9D140225A719A792D
:1085000002F00C02082AFAD1064B9A795206FBD5E2
:1085100022221A709A7902F00C020C2AFAD17047C2
:1085200000700440004006400000330100001301C9
:1085300000500640184B5A7902F0E0025A711A793D
:1085400002F0F8021A71A3F55B33A3F570731A6891
:1085500042F004021A60114A136823F0784323F0B2
:10856000010313600E4B1A7802F08C0242F05002A5
:108570001A705A7802F09C0242F040025A709A78BF
:1085800002F0E6029A70074A00231370064A82F846
:10859000353383F31188704700F0074000D0004066
:1085A00000D0074000E0074000E100E0104B6846C3
:1085B0001A6820F0070101328D4601B51A600D4B93
:1085C0001A6801321A600C4B1A683AB11A68013AFB
:1085D0001A601B6813B9094B01221A70084B1A68FC
:1085E00012B11A68013A1A60BDE801408546704729
:1085F0001C86FF1F5C98FF1FA893FF1FA493FF1FFB
:10860000AC93FF1F024B034A5A6007221A6070475F
:1086100010E000E000770100014B1868704700BFD0
:108620001C86FF1F072888BF0020134B134A53F8EE
:10863000203010B5124CB4FBF3F441F22803422071
:10864000D15841F48061D1500E4B4FF440729A637F
:10865000DA6305F001FF0C4B0022DA709A709A7110
:10866000DA725A71C4F30422E4B21A705C70DA78D8
:1086700042F02C02DA7010BD28170100007004408F
:10868000C0C62D0000B0044000A00E40094B1A687F
:1086900059680132202A08BF00228A4208D019688E
:1086A000194408721A60044BDA7842F08002DA70DA
:1086B000704700BF2086FF1F00A00E400A4B996A3A
:1086C000DA6A91420CD09A6A511C1A44996292F863
:1086D000302002709A6A202A04D100229A6201E0B6
:1086E00000207047012070472086FF1F044B1A7836
:1086F00002F0FF0012B100221A700120704700BF83
:10870000A493FF1F014B1865704700BF2086FF1F11
:10871000684620F007018D4631B527480179C9B276
:108720008C0615D5254BDA6A9C6A0132202A08BFCF
:108730000022A24206D0DD6AC4795819E4B280F85A
:108740003040DA621E4A052010601A6D1D4B1A6017
:108750004A0608D51C4B4FF480529A60164BDA78C3
:1087600002F0BF02DA700B0621D5164B1968F1B979
:10877000124B18685A68904214D0134A4FF4805034
:1087800050605A68501C1A445860107A0A4AC0B2A5
:10879000D0715868202808BF5960D37843F040034F
:1087A000D37004E0044BDA7802F07F02DA70BDE89F
:1087B00031408546704700BF00A00E402086FF1F55
:1087C000A893FF1FAC93FF1F80F00F4062B6704765
:1087D00072B6704762B6704772B670474FF0E023CA
:1087E00008B1034A00E0034AC3F80C2D704700BFEC
:1087F0000400FA050100FA0513B53F4A3F484FF45B
:1088000080730E214360836091605161A2F535222F
:108810004FF4F00153629364D36413655365936519
:1088200002F53522403251619160354A4FF4907122
:1088300051621363936402F5342280324FF49051F5
:1088400091604FF48021516001F5905151612D4AA2
:1088500040F20311116051609160D160116151616A
:108860009161D16102F53322C03200245461264A5D
:108870002649136153619361936602F5322202F532
:1088800080729160516103600A21C36022462346D1
:1088900019480824446000240194019CB4F57A7FAF
:1088A00002D2019C0134F7E70069C40712484FF077
:1088B0000804846048BF013200240194019CB4F58F
:1088C0007A7F02D2019C0134F7E70069C00758BFE4
:1088D00001330139DCD10A2A0D4A03D10A2B01D117
:1088E000012300E000231370044B4FF4E0621A6090
:1088F000DA6002B010BD00BF00F00F4000900440ED
:1089000000B0044000C0044000D0044070000004E7
:10891000E293FF1F104B1B7882B0D3B10F4B0222A2
:108920009A6004225A600022019201990C4A9142F5
:1089300002D8019A0132F7E702225A6004229A60B3
:1089400000230193019A064B9A42E7D8019B013319
:10895000F7E702B0704700BFE293FF1F00F00F403F
:108960001FA1070003280DD8DFE800F00204060865
:10897000102205E0202203E0402201E04FF0806257
:10898000014B5A60704700BF00F10F4003280DD81B
:10899000DFE800F002040608102205E0202203E0D0
:1089A000402201E04FF08062014B9A60704700BFA7
:1089B00000F10F4038B50546002445FA04F3DB0703
:1089C000E0B202D5FFF7CEFF01E0FFF7DFFF013491
:1089D000082CF2D138BD08B5032813D8DFE800F021
:1089E00002040608002004E0012002E0022000E06A
:1089F000032004F00FFB43F27C03984294BF002055
:108A0000012008BD002008BD032817D8DFE800F0CA
:108A100002070C110A4B1868C0F300107047084B8E
:108A20001868C0F340107047054B1868C0F38010F9
:108A30007047034B1868C0F3806070470020704790
:108A400000F10F4038B500242546E0B2FFF7C3FF20
:108A500018B10123A3401D43EDB20134082CF4D119
:108A6000284638BD024B1869C043C0B2704700BFEA
:108A7000C0F00F4008B5082004F0CCFA5E2804D9F5
:108A8000104B1A784AB9012206E0082004F0C2FA15
:108A9000542802D80B4B00221A70082004F0BAFAAE
:108AA000632804D9084B4FF400725A6008BD0820AF
:108AB00004F0B0FA542803D8034B4FF400729A60C4
:108AC00008BD00BF7486FF1F80F00F40034B18786D
:108AD000013801288CBF0020012070477486FF1FD9
:108AE000034B1878012806BF02221A700020704735
:108AF0007486FF1FC0B205F0FFBAC0B205F0EABA33
:108B00000B4B10F0010F4FF4800214BF5A609A60B3
:108B100010F0020F4FF4001214BF5A609A6010F068
:108B2000040F4FF4801214BF5A609A60704700BF60
:108B300040F00F4008B507F0CFFB05F097FE05F0B9
:108B400047FEBDE8084007F049BC38B5054605F0CA
:108B500095FD08280AD900242819013405F00EFED5
:108B6000092CF9D105F03EFE012038BD002038BDAA
:108B7000092105F0A3BD002006F02CB8224A41F2DD
:108B80003C030120D15841F44051D1501F4B2049A2
:108B900018601A680A431A601E4ADA601A61DA6AB3
:108BA00042F08052DA621A6822F001021A601A68F2
:108BB00022F000621A60184A4FF400731360536089
:108BC0009360D360136153619361D361A2F5F03276
:108BD00010601068014311601049D16001F5200157
:108BE0001161D16A41F08051D162116821F0010117
:108BF0001160116821F00061116002F5E8329362A2
:108C0000D3621364536470470070044000C0024094
:108C1000000C1F800300013E00B004400400513EE0
:108C2000FF2800F03F031AD82C4872B141F00061D0
:108C300041EA03434363294BDA6A002A1946FADA08
:108C4000CA6A264BD200FBD541E041F0004141EA1F
:108C500003434363214BDA6A002AFBDA37E0B0F5BD
:108C6000007F1AD21E4872B141F0006141EA03430D
:108C700043631B4BDA6A002A1946FADACA6A184BB0
:108C8000D000FBD523E041F0004141EA03434363B8
:108C9000134BDA6A002AFBDA19E0124872B141F08C
:108CA000006141EA034343630E4BDA6A002A194626
:108CB000FADACA6A0B4BD200FBD508E041F000415A
:108CC00041EA03434363074BDA6A002AFBDA986BF5
:108CD000DA6A42F01042C0B2DA62704700C0024065
:108CE00000D0024000C00A4010B5FFF795FC0446D2
:108CF000FFF792FC001B0028B8BF40420628F7DDB2
:108D000010BD07B5030A8DF805008DF80610032283
:108D100001A9A0208DF8043004F0A0FBFFF7E4FFC8
:108D200003B05DF804FB2DE9F04100238AB08846CA
:108D300016461C46B4421DD00AAA1A445D1C18F8F7
:108D4000041002F8221C2F18FA0602D0721E944258
:108D50000DD1020A8DF804208DF8050001A9DA1C56
:108D6000A02004F07BFB0025FFF7BEFF384601344E
:108D70002B46DFE70AB0BDE8F0811FB5030A0222E7
:108D800003A98DF80C308DF80D0000920B46A02041
:108D900004F0B8FB9DF80C0005B05DF804FB1FB5AE
:108DA0000B46010A8DF80C108DF80D00009203A9F6
:108DB0000222A02004F0A6FB05B05DF804FBC0EB86
:108DC000C00000F5B0400722FFF7ADBFC0EBC00008
:108DD00000F5B0400722FFF7E2BF30B500238BB0AB
:108DE00001AD00225A550133222BF9D14FF4B04482
:108DF000230A8DF8054029462222A02020348DF830
:108E0000043004F02BFBFFF76FFFB4F5803FEFD188
:108E10000BB030BD13B50C46C0EBC000072200F507
:108E2000B0406946FFF7BBFF9DF8002023789A42C7
:108E300011D19DF8012063789A420CD19DF802204F
:108E4000A3789A4207D1DDF80300D4F80330C31A9F
:108E50005842584100E0002002B010BD704713B5E1
:108E600045F2FF70FFF789FF552802D1254B1B788B
:108E7000B3B345F2FF700021FFF743FFFFF7ADFFEB
:108E8000002021494022FFF74EFF402420461F4981
:108E900040224034FFF747FFB4F5E07FF6D10023CE
:108EA00001934FF4D364204601A90422FFF73BFF4E
:108EB000043440F678039C42F5D1002301934FF42B
:108EC000FF64204601A90422FFF72DFF043440F679
:108ED000D8039C42F5D145F2FF705521FFF711FFF1
:108EE000002009494022FFF75AFF40240849204644
:108EF000214440224034FFF752FFB4F5E07FF5D122
:108F000002B010BDE293FF1F0C80FF1F5817010035
:108F1000B893FF1FF7B5CE4EB4787278052C35465E
:108F200000F29784A22A00F0848300F2B780132A0B
:108F300000F0A38242D8072A00F0E9811AD8022A59
:108F400000F062810CD8002A00F04F81012A40F025
:108F5000828404F001032021994041F001014AE19B
:108F6000052A00F0A38100F2BB81042A00F0788179
:108F700000F071BC0F2A00F0568209D80D2A00F0CB
:108F80000A8200F22C820C2A00F0E18100F063BC1E
:108F9000112A4FEA540604F00107AE4B00F052824A
:108FA00000F25E8253F82430D5F803009847202160
:108FB00001FA07F7024647F005014FE21A2A00F0CE
:108FC000D38226D8162A00F074820CD8142A00F016
:108FD0006282152A40F03F8404F001032021994069
:108FE00041F00C0107E1182A4FEA540604F001078A
:108FF00000F06D8200F28D82964BD5F8030053F895
:1090000024309847202101FA07F7024647F0130160
:1090100024E2202A00F0DE8224D81C2A00F0D1822B
:10902000C0F0C6821F2A40F0168404F001012026F9
:1090300006FA01F141F010016008C9B204F000FB2A
:10904000AA78EB7802F001018E40C0F3072446F0C5
:109050001001C0B2019000945008C9B2002203F080
:109060000F0371E17F2A00F0CD828C2A00F0D682B6
:10907000212A40F0F08304F00101090141F06E0162
:10908000600804F0DDFAB378F278009203F0010191
:109090000901C0B241F06E010190AEE2B52A00F0C4
:1090A0004B8340D8A92A00F0118318D8A52A00F0D4
:1090B000D2820ED8A32A00F0C582A42A40F0CB8326
:1090C000D6F803102046C9B203B0BDE8F04004F062
:1090D00029BCA72A00F0E88240F2D282EDE2AD2A54
:1090E00000F00F830DD8AB2A00F0F98200F2008364
:1090F000D6F803102046C9B203B0BDE8F04004F032
:1091000080BDB12A00F00683B32A00F00C83AE2A9A
:1091100040F0A183D6F803102046C9B203B0BDE8E1
:10912000F04004F09FBDC32A00F049832BD8BB2A2E
:1091300000F0228316D8B82A00F00C83B92A00F078
:109140001283B62A40F08783424BD6F8030053F8C7
:109150002430984704F0010320219940024641F051
:109160001101F4E2C12A00F0198300F21E83BC2A27
:1091700040F07183D6F803102046C9B203B0BDE8B1
:10918000F04004F081BED12A00F02B831DD8CA2AFA
:1091900000F02083CC2A00F0F882C92A40F05B83DB
:1091A0006008182104F04CFA00F48064B0782021A3
:1091B00000F001029140D6F8032041F0180122F49A
:1091C00080624008C9B2224319E0D42A00F0178314
:1091D000FF2A00F01B83D22A40F03D831E4BD6F8B5
:1091E000032003EB8413DA6103E304F0010320217D
:1091F000994041F00D01D5F803206008C9B203B0D1
:10920000BDE8F04004F0ECB9D6F803306008002B5C
:1092100004F001044FF0200303FA04F1C8BF012257
:10922000C9B204F0DDF9B4780C4BD6F80300012282
:109230001A55084B0028B8BF404253F824309847CD
:1092400004F0010320219940024641F007017EE22B
:109250004896FF1F7886FF1FF893FF1FDA93FF1FC2
:10926000BD4ED5F8030056F824300028B8BF404260
:10927000984706EB8404A061A878202400F001013F
:1092800004FA01F14008C9B204F0DAF9002840F00C
:10929000E582B24B987800F0010106EB80068C4025
:1092A00044F007014008C9B2B269A8E7AC4BD6F850
:1092B000030000221A55A84B03EB84031B6B98474D
:1092C000B378A84A03F0010142F82400202000FAF4
:1092D00001F141F006015808C9B252F823208EE787
:1092E000202604F0010106FA01F141F01001C9B293
:1092F000600804F0A5F90346A878EA7800F00101B7
:10930000D2088E40009246F01001DAB216E0202515
:1093100004F0010105FA01F141F01001C9B2600841
:1093200004F08EF90346C3F30722B078009200F0F0
:109330000101F2788D4045F01001D20801924008F9
:10934000C9B20022C3F3074304F00EF986E204F029
:109350000101202606FA01F141F01401C9B26008AA
:1093600004F06EF9D5F803100246A87849B900F068
:1093700001018E4046F014014008C9B242F00202D9
:109380003DE700F001018E4046F014014008C9B2EB
:1093900022F0020233E704F00101202606FA01F16F
:1093A00041F01401C9B2600804F04AF9D5F803107D
:1093B0000246A87849B900F001018E4046F0140138
:1093C0004008C9B242F0010219E700F001018E40E5
:1093D00046F014014008C9B222F001020FE704F080
:1093E0000101202606FA01F141F01401C9B260081A
:1093F00004F026F9D5F803100246A87849B100F028
:1094000001018E4046F014014008C9B242F010023A
:10941000F5E600F001018E4046F014014008C9B2A3
:1094200022F01002EBE64C4BD6F8030003EB84036A
:109430001B6B984704F0010320219940024641F03C
:10944000040184E103EB8404D5F80300236B9847FF
:10945000202101FA07F7024647F00801304677E17C
:1094600003EB8404D5F80300236B9847202101FA0D
:1094700007F7024647F00A01F0E7374BD6F803003A
:1094800053F82430984704F0010320219940024604
:1094900041F003015BE1304BD6F8030053F8243070
:1094A000984704F0010320219940024641F00B0146
:1094B0004DE1294BD6F8030053F82430984704F0C7
:1094C000010320219940024641F012013FE120248E
:1094D00004FA07F747F01401C9B2304604F0B0F8B7
:1094E000D5F803100246A87849B100F001018C407C
:1094F00044F014014008C9B242F008027FE600F0CF
:1095000001018C4044F014014008C9B222F0080265
:1095100075E6202404FA07F747F01401C9B2304673
:1095200004F08EF8D5F803100246A87849B100F08F
:1095300001018C4044F014014008C9B242F0040219
:109540005DE600F001018C4044F014014008C9B20E
:1095500022F0040253E600BF7886FF1F4896FF1FE3
:109560004096FF1F2896FF1F04F00101202505FAF1
:1095700001F141F01401C9B2600804F061F8D6F8B5
:1095800003100246B07849B100F001018D4045F06A
:1095900014014008C9B242F4006230E600F0010153
:1095A0008D4045F014014008C9B222F4006226E65D
:1095B000D6F803102046C9B203B0BDE8F04004F06D
:1095C0004DB9D6F803102046C9B203B0BDE8F0404B
:1095D00004F05DB904F00101090141F06E01600879
:1095E00004F02EF8B378C0F3072003F001010090D7
:1095F0000901F278019241F06E0100225808C9B2C7
:109600001346A1E6D6F80330022B00F22281944BD8
:109610001C44944BDB7884F848301FE1D6F80310E3
:10962000C1F108012046C9B203B0BDE8F04004F022
:10963000E3B8D6F803102046C9B203B0BDE8F04045
:1096400004F0A8B8D6F803102046C9B203B0BDE8AC
:10965000F04004F035B9204604F04EFAB378D6F85D
:10966000031030B91846C9B203B0BDE8F04004F0A9
:1096700078B81846C9B203B0BDE8F04004F06BB941
:10968000204604F039FAD6F8031030B9B078C9B2E0
:1096900003B0BDE8F04004F04BB8B078C9B203B0F5
:1096A000BDE8F04004F077B9D6F803102046C9B2FF
:1096B00003B0BDE8F04004F01BB8D6F80310204614
:1096C000C9B203B0BDE8F04004F0E3BAD6F8031025
:1096D0002046C9B203B0BDE8F04004F079BAD6F82C
:1096E00003102046C9B203B0BDE8F04004F057BAF9
:1096F000D6F803102046C9B203B0BDE8F04004F02C
:1097000099BAD6F803102046C9B203B0BDE8F040BC
:1097100004F0D8BAD6F803102046C9B203B0BDE8A9
:10972000F04004F082B8D6F803102046C9B203B066
:10973000BDE8F04004F048B9494BD6F8030053F8AF
:1097400024309847484B03EB8414206186E060087E
:10975000C9B254E5D6F803102046C9B203B0BDE83B
:10976000F04004F0C6B8D6F803102046C9B203B0E2
:10977000BDE8F04004F027B8D6F803102046C9B27F
:1097800003B0BDE8F04004F066BBD6F803102046F5
:10979000C9B203B0BDE8F04004F00CBB324B03EBA0
:1097A0008414D6F80330237258E02D4BD6F803000A
:1097B00053F824309847A4012B4B18514EE0284B06
:1097C000D6F8030053F824309847274B03EB841452
:1097D000606043E0244BD6F8032003EB84135A83E4
:1097E00007E0D6F80310204603B0BDE8F04004F0CF
:1097F0000DBE204603B0BDE8F04004F044BD1A4B56
:1098000003EB8414D6F80330236227E0D6F8033044
:109810008BB1012B1DD1144A02EB84121376104B2D
:10982000124A43F8242003EB8404114B2365114BA7
:109830002363114B0BE00C4A02EB84121376084AA7
:109840000E4B42F8243002EB840423652363A366A5
:1098500004E0042200E00322094B1A7003B0F0BDBB
:109860007886FF1F4896FF1FF893FF1F8DE10000C9
:10987000F1E10000C9E1000031E2000059E200001E
:109880006098FF1F38B5D44DD44CA8786B78052864
:1098900002D90423237038BDA32B00F05B8200F2B1
:1098A000BE80112B00F0E2814FD8082B00F07F81A1
:1098B00029D8032B00F04F810ED8012B4FEA50021C
:1098C00000F0010100F0328100F23B81202303FA15
:1098D00001F141F00D012EE1052B00F05281C0F0A5
:1098E0004A81062B00F05581072B40F0E98200F0F9
:1098F00001032021994041F010014008C9B203F052
:109900009FFEC0B251E10C2B00F0798107D80A2BE1
:1099100000F05A8100F26C8104F026FC0FE10E2B5E
:1099200000F08C81C0F07B810F2B00F09481102B14
:1099300040F0C682AA4B03EB800320211D6D00F08E
:109940000103994041F005010FE11A2B00F0D48189
:109950002FD8152B00F0A68113D8132B4FEA5002F5
:1099600000F001019E4D4FEA800000F08A8100F274
:1099700091812844202303FA01F1856E41F00A0108
:1099800086E1172B00F0A081C0F09381182B00F026
:10999000A681192B40F0948200F001032021994008
:1099A00041F014014008C9B203F04AFEC0F3800040
:1099B000C5E0202B00F0BA8117D81C2B00F0AC8139
:1099C000C0F0A7811D2B00F0AA811F2B40F07882E8
:1099D00000F001032021994041F010014008C9B274
:1099E00003F02EFEC0F30340A9E07F2B00F0A88116
:1099F0000CD8212B40F0648200F0010109014008DD
:109A000041F06E0103F01CFE001298E08C2B00F078
:109A10009C81A22B40F0548204F020F88FE0B92BF7
:109A200000F0E8813AD8AC2B00F0B98119D8A72B07
:109A300000F0A98107D8A52B00F08F8100F2988152
:109A400004F074F87BE0A92B00F0A381C0F09E81A4
:109A5000AA2B00F0A181AB2B40F0328204F04BF92D
:109A60006DE0B32B00F0A4810AD8AE2B00F09D81ED
:109A7000C0F09881B12B40F0238204F016F85EE02C
:109A8000B52B00F0A381C0F09681B62B00F0A78122
:109A9000B82B40F0158204F03CF850E0C92B00F0E0
:109AA000CD811CD8C12B00F0AE810BD8BC2B00F0AF
:109AB000A481BD2B00F0A481BB2B40F0018204F0F7
:109AC00020FA3CE0C32B00F0AB81C0F0A181C42B95
:109AD00000F0B081C52B40F0F381424BABE1D02BBD
:109AE00000F0D68112D8CC2B00F0B08107D8CA2B59
:109AF00040F0E6813C4B03EB8010438BDEE1CE2B44
:109B000000F0A781CF2B00F0AF81D9E1D22B00F07C
:109B1000CC81C0F0C781D42B00F0CC81FF2B40F06A
:109B2000CF81314B03EB8010037EC7E1202303FA82
:109B300001F141F001011046C9B203F081FD6060FE
:109B4000C0E1274B03EB8000202303FA01F1056DF0
:109B500041F007019CE0224B03EB800320211D6DA7
:109B600000F00103994041F002014008C9B203F03E
:109B700067FDA847E3E71A4B03EB8000036D80699C
:109B800056E1174B194A03EB800352F820009B6EF5
:109B90004EE100F001032021994041F010014008FE
:109BA000C9B203F04DFDC0F30720C000C7E700F0C5
:109BB00001032021994041F015014008C9B203F08A
:109BC0003FFDC0F34020BAE700F001032021994097
:109BD00041F0150119E000BF4896FF1F6098FF1F74
:109BE0007886FF1F7C95FF1FF893FF1F2896FF1FA5
:109BF00000F001032021994041F0150115E000F02B
:109C000001032021994041F014014008C9B203F03A
:109C100017FD10F0020F14BF002301234EE100F0E6
:109C200001032021994041F014014008C9B203F01A
:109C300007FD00F0010080F0010080E700F0010363
:109C40002021994041F014014008C9B203F0F8FC0A
:109C5000C0F3001073E7A44B03EB800320219D6E3B
:109C600000F00103994041F004017EE79E4B03EBB5
:109C7000800320219D6E00F00103994041F008010E
:109C800073E72844202303FA01F1056D41F0030135
:109C900010466BE72844202303FA01F1056D41F0DB
:109CA0000B01F5E700F001032021994041F00C0180
:109CB000CAE08D4B03EB800320211D6D00F00103F2
:109CC000994041F0120150E7874B03EB80032021BC
:109CD0001D6D00F00103994041F0130145E700F0CC
:109CE00001032021994041F014014008C9B203F05A
:109CF000A7FCC0F3C00022E700F001032021994037
:109D000041F014014008C9B203F09AFCC0F3C0202E
:109D100015E703F0D7FE12E703F0E1FE0FE7724B01
:109D200003EB80031D6D02F09BFB22E700F00101B5
:109D30000901400841F06E0103F082FCC0B2FEE66A
:109D4000694B184490F84830B8E003F0A1FEC0F128
:109D50000800F4E603F0D0FEF1E603F0CDFE18B9FA
:109D6000A87803F06EFEEAE6A87803F0ECFEE6E6DB
:109D700003F0C2FE18B9A87803F056FEDFE6A87813
:109D800003F0F3FEDBE603F038FED8E603F0F8FF5D
:109D9000D5E603F0BDFFD2E603F0C7FFCFE603F040
:109DA000D1FFCCE603F0F9FFC9E603F0D8FFC6E621
:109DB00003F0E8FEC3E600F001010901400841F0AC
:109DC0006F0103F03DFCC0F30440B8E6464B474A40
:109DD00003EB800302EB80101B6D006928E0424B0F
:109DE00003EB800320211D6D00F00103994041F039
:109DF0001101BAE603F03FFEA1E604F08EF89EE6FC
:109E000004F096F89BE6394B03EB8010037A55E09B
:109E1000354B364A03EB800380011B6D105807E079
:109E2000314B324A03EB800302EB80101B6D40681C
:109E3000984784E62E4B53F820303FE000F00103B2
:109E40002021994041F01801400875E604F035F8EA
:109E500075E600F001010901400841F06F0103F0CF
:109E6000EFFBC0F309006AE6AB78224AD05C002120
:109E7000616010B1204801254560D1541F4AD15C72
:109E800019B1616841F0020161600021D15419E00B
:109E900000F001010901400841F06F0103F0D0FB1F
:109EA00000164CE604F0A8FA49E6104B03EB8010CC
:109EB000C36903E00D4B03EB8010036A636001E0AC
:109EC000032323700E4B1B7863B10E4B62681A603C
:109ED0000D4B1AB91A6842F0080202E01A6822F023
:109EE00008021A6038BD00BF7886FF1FF893FF1F75
:109EF000B493FF1FF093FF1F6098FF1FD493FF1FC1
:109F00005B98FF1F4C98FF1F5096FF1F38B5A94A5A
:109F10009378022B144600F00681032B00F00A818F
:109F2000002B40F0078253784E2B00F0A5802BD8F1
:109F3000462B75D016D8422B63D009D8402B5CD065
:109F4000412B40F0F5819C4BD178197000205CE0EA
:109F5000442B5ED0452B40F0EB81974BD178597163
:109F6000052052E04B2B77D004D8472B60D0492BEB
:109F700066D0DDE14C2B7AD04D2B40F0D9818E4B51
:109F8000D1785975152040E0542B00F0A6801BD8DD
:109F9000512B00F0828009D84F2B77D0502B40F006
:109FA000C781854BD178997516202EE0522B00F091
:109FB0008380532B40F0BC817F4DD2F8033029467B
:109FC000102041F8103F7EE0842B00F0A1800BD8D8
:109FD000552B00F08D80832B40F0AA81774BD2F86F
:109FE0000320C3F8802038BD852B00F09680FF2B1E
:109FF00040F09E81D278724B9EE145F2FF70D1789D
:10A0000003E06D4BD17859700120BDE83840FEF770
:10A0100078BE6949D2F8033041F81C3F1C2005E0A6
:10A020006549D2F8033041F80C3F0C2004226BE064
:10A03000614DD2F803302946082041F8083F42E03C
:10A04000D2785D4B0AB9DA7503E05E490122DA7510
:10A050004A601720D97DD8E7574CD178E1700320AA
:10A06000FEF74FFEE078BDE83840FEF74BBB524BA1
:10A07000D17899700220C8E74F4CD2F80300E084F1
:10A08000FEF73EFD2620211802223DE0D2F8031003
:10A09000494BC9B259761920B7E7474B1A7D12F0E0
:10A0A000010F1D4604D0E378DB0701D4FEF795FECF
:10A0B000E17829751420A8E73F49D2F8033041F828
:10A0C000203F2020B2E70422FEF72DFE687929897F
:10A0D0002A8ABDE8384002F0CDBFD2F80330012B08
:10A0E00000F228813449D37801F81A3F1A200AE097
:10A0F000D2F80330012B00F21D812E4B2E49DB7864
:10A1000001F81B3F1B200122BDE83840FEF70BBEC3
:10A110002D4BD2F803201A6038BD284BD2F803200B
:10A12000C3F8842038BD5178284BD2F8032043F877
:10A13000212038BD53782E2B00F2FA80DFE813F08F
:10A140002F004A005400F800F800F800F800F8006A
:10A15000F8005E00630068006D0072007700F80090
:10A16000F800F800F800F800F800F800F800F8002F
:10A17000F800F800F8007C0083008A009100980045
:10A180009F00A600AD00B400BB00C200C900D00013
:10A19000D500DA00DF00E400E900EE00F3000C4B2C
:10A1A000D4F803201A60FEF737FA044BC3F888008E
:10A1B00038BD00BF4896FF1F0C80FF1F7886FF1F29
:10A1C0005A98FF1F6098FF1F5C98FF1F6C98FF1F35
:10A1D0009495FF1F594BD4F803205A60FEF71CFAE0
:10A1E000574BC3F88C0038BD544BD4F803209A6009
:10A1F000FEF712FA524BC3F8900038BD4F4BD4F81B
:10A200000320DA6038BD4D4BD4F803201A6138BD05
:10A210004A4BD4F803205A6138BD484BD4F8032088
:10A220009A6138BD454BD4F80320DA6138BD434B01
:10A23000D4F803201A6238BDD4F803203F4BD2B2C1
:10A2400083F8242038BDD4F803203C4BD2B283F8E5
:10A250002A2038BDD4F80320384BD2B283F8252009
:10A2600038BDD4F80320354BD2B283F82B2038BD4B
:10A27000D4F80320314BD2B283F8262038BDD4F86D
:10A2800003202E4BD2B283F82C2038BDD4F8032003
:10A290002A4BD2B283F8272038BDD4F80320274BAD
:10A2A000D2B283F82D2038BDD4F80320234BD2B28C
:10A2B00083F8282038BDD4F80320204BD2B283F88D
:10A2C0002E2038BDD4F803201C4BD2B283F82920AD
:10A2D00038BDD4F80320194BD2B283F82F2038BDF3
:10A2E000164BD4F803201A6338BD144BD4F803205E
:10A2F0005A6338BD114BD4F803209A6338BD0F4B15
:10A30000D4F80320DA6338BD0C4BD4F803201A6468
:10A3100038BD0A4BD4F803205A6438BD074BD4F833
:10A3200003209A6438BD054BD4F80320DA6438BDA5
:10A33000032200E00422034B1A7038BD9495FF1FDE
:10A340007886FF1F6098FF1F2DE9FF41C64EC74F5B
:10A3500032787A7064233B70212AD6F803307B6010
:10A3600035463C4601F092805AD80E2A00F0CA8445
:10A370002AD8072A00F03D8311D8032A00F08881EB
:10A3800007D8012A00F0BE80022A00F0118101F0F6
:10A390006BBB052A00F0258340F2A58125E30A2A3C
:10A3A00000F02F8309D8082A00F02383092A41F0FE
:10A3B0005B83FFF7ABFD01F059BB0C2A00F05D8415
:10A3C00040F2448400F06FBC182A00F0098612D8CD
:10A3D000142A00F02D8507D80F2A00F0B284132A22
:10A3E00000F0ED8401F040BB162A00F0E18540F258
:10A3F0004F8500F0E2BD1C2A00F0408706D81A2ADB
:10A4000000F0108640F2FD8500F01DBE1F2A00F00E
:10A41000898700F2D4871E2A00F0358701F024BB1B
:10A42000802A01F01F8138D8402A01F009811BD809
:10A43000242A01F094800DD8222A01F08980232A51
:10A4400041F012838A4B1B68C6F80330FFF75EFDAC
:10A4500001F00CBB262A01F0B980C1F0AD80272A9B
:10A4600001F0DC8001F000BB442A01F0F28008D842
:10A47000422A01F0E88001F2E98001F0EAFF01F0F0
:10A48000F5BA462A01F0EB80C1F0E680472A41F098
:10A49000EB8201F0E4FF01F0E9BA872A01F0B48110
:10A4A00017D8832A01F0FA800BD8812A01F0DF80C7
:10A4B000822A41F0D9826F4B022283F8942001F066
:10A4C000D5BA852A01F01D816B4A41F2098101F05C
:10A4D0002BB98C2A01F0F08109D8892A01F0BE81BC
:10A4E000C1F05D818A2A01F0D08101F0BDBAF22A63
:10A4F00001F06C82FF2A01F0AE828D2A41F0B48215
:10A5000001F0FEB9B378052B55D85C4A5C4E0024A7
:10A51000D4545C4AD454F25C72B103F0010220219D
:10A520009140594A41F00601580852F82320C9B217
:10A5300003F056F8AB78F454AC78544BD5F80300DC
:10A5400001271F554B4B0028B8BF404253F8243019
:10A550009847202604EA070106FA01F141F00701B5
:10A560000246C9B224FA07F003F03AF8D5F80330EE
:10A57000A878002B0DDD00EA070306FA03F100229C
:10A580008DE88400F840C9B2134602F0EDFF01F0F7
:10A590006DBA00F0010306FA03F1002202238DE8F0
:10A5A0000C004008C9B2134602F0DEFF01F05EBAAB
:10A5B000B378052B03D90423237001F057BA2F4A2F
:10A5C0002F4E0024D4542F4AD454F25C7AB103F0B5
:10A5D0000102202191402C4A41F00601580852F80E
:10A5E0002320C9B202F0FCFF1F4B9B78F454AC78D7
:10A5F000264BD5F8030001271F551E4B0028B8BF76
:10A60000404253F824309847202604EA070106FA0E
:10A6100001F141F007010246C9B224FA07F002F045
:10A62000DFFFD5F80330A878002B0EDD00EA070322
:10A6300006FA03F1002202238DE80C00F840C9B2AB
:10A64000134602F091FF01F011BA00F0010306FA7F
:10A6500003F100228DE884004008C9B2134602F0DD
:10A6600083FF01F003BA00BF4896FF1F6098FF1FE9
:10A670004C98FF1F7886FF1F0C80FF1FD493FF1F8D
:10A680004096FF1FF093FF1F2896FF1FDA93FF1FCE
:10A69000B07805288FD802F01BFCB0789D4B0122C2
:10A6A00000EA0201202404FA01F141F007011A54E2
:10A6B000C9B2D040002202F093FFB07800F001014F
:10A6C00004FA01F102230024019322462346009458
:10A6D0004008C9B202F048FFB3788F4AD4548F4A79
:10A6E000D45401F0C3B9B078052804D98C4A527803
:10A6F000022A41F0BB81884A894F00261654874AB6
:10A7000016546A78012A49D003D3022A00F0AF8098
:10A7100063E1804C235C7BB100F001032021994070
:10A72000804B03EB800341F007019A694008C9B2EE
:10A7300002F056FFBB78E654AB787B4CE25C82B10A
:10A7400003F0010220219140784A41F0060152F8BD
:10A7500023205808C9B202F043FF714B9B780022B6
:10A76000E254A878D5F80320202400F0010104FA6F
:10A7700001F141F00D014008C9B202F031FFA878A3
:10A7800000F00103002204FA03F100920192400854
:10A79000C9B2134602F0E8FE01F068B9614A131825
:10A7A000904693F84830012B0CD004D3022B14D1DF
:10A7B00003F022FE10E000F001032021994041F057
:10A7C0000D0105E000F001032021994041F0010155
:10A7D0004008C9B202F034FF0646A8784D4F3B5CF2
:10A7E00083B100F001032021994008EB800341F080
:10A7F00007019A694008C9B202F0F2FE484B9B7803
:10A800000022FA54AB78484FFA5C82B103F001029F
:10A8100020219140454A41F0060152F82320580872
:10A82000C9B202F0DDFE3E4B9B780022FA54A878B4
:10A83000D5F8033000F00101202707FA01F11E448A
:10A8400041F00D014008C9B2324602F0C9FEA878B5
:10A8500000F00103002207FA03F100920192400880
:10A86000C9B2134602F080FE666001F0FFB8142BF7
:10A8700000F3AF8003065FD53446AB782341DF0792
:10A8800042D5DFF8908014F80830670804F001061C
:10A890006BB12021264BB14041F0070153F8242031
:10A8A000F8B2C9B202F09CFE002304F80830DFF8C9
:10A8B000788014F808306BB120211C4BB14041F076
:10A8C000060153F82420F8B2C9B202F089FE002331
:10A8D00004F80830202303FA06F6D5F803300622E0
:10A8E00002FB0342134BFFB246F00D0153F8222046
:10A8F0003846C9B202F074FE002200920192384636
:10A90000F1B2134602F030FE0134062CB5D101F04D
:10A91000ADB800BFDA93FF1FD493FF1FF093FF1F62
:10A920004896FF1F7886FF1F4096FF1F2896FF1F3F
:10A930009086FF1F5496FF1F05284AD8A44C235C1D
:10A940007BB100F0010320219940A24B03EB80036F
:10A9500041F007019A694008C9B202F041FEBB7894
:10A96000E654AB789C4CE25C82B103F001022021FA
:10A9700091409A4A41F0060152F823205808C9B282
:10A9800002F02EFE964B9B780022E254A878D5F870
:10A990000330202400F00101062202FB030204FA26
:10A9A00001F1904B41F00D0153F822204008C9B24B
:10A9B00002F016FEA87800F00103002204FA03F169
:10A9C000009201924008C9B2134602F0CDFD01F099
:10A9D0004DB80423237001F049B80323237001F01C
:10A9E00045B8FEF797FA01F041B8FEF74BFF01F0CA
:10A9F0003DB8B378052B3FF6DEAD0323237001F09D
:10AA000035B8B378022B00F0AC80032B00F0AE8099
:10AA1000002B40F003817378502B71D027D8472B3F
:10AA200062D013D8422B55D007D8402B4CD0412BA5
:10AA300040F0F2806C4B1B784EE0452B4ED050D846
:10AA4000442B40F0E980684BDB6945E04C2B50D04B
:10AA500007D8492B4AD04B2B40F0DE80624BDB7885
:10AA60003AE04E2B604B47D048D85B7D34E0802BDA
:10AA700055D014D8532B49D007D8512B43D0522B43
:10AA800040F0CA80584B1B6A26E0552B44D040D377
:10AA9000562B40F0C180544B93F824301CE0832B9C
:10AAA00048D008D8812B3ED0822B40F0B580494B4E
:10AAB000D3F8983010E0852B42D03FD3FF2B40F0E5
:10AAC000AB804A4B1B7848E045F2FF70FEF755F922
:10AAD0007860A5E0444B5B786360A1E0424B5B7912
:10AAE000FAE7414BDB68F7E73F4B6BE03E4BDB7D22
:10AAF00033E03D4B9B78EFE7DB8CEDE75B7EEBE7EC
:10AB0000394B9B7DE8E7384B1B7DE5E7364B1B69EE
:10AB1000E2E7354B9B7EDFE7334BDB7EDCE72D4BFB
:10AB200093F89430D8E72B4B93F894301E1F734260
:10AB30007341D1E7274BD3F88030CDE72C4B3EE073
:10AB4000244A2C49D2F884304B4303F5405339331F
:10AB5000C2F8843023F00043BEE7003318BF01235E
:10AB6000BAE77278244B53F82230B5E77378282B74
:10AB70002AD011D8022B24D005D8FBB1012B4BD100
:10AB80001E4B5B68A8E7092B46D30E2B48D9272B11
:10AB900042D11A4B1B6B9FE72B2B34D006D8292BA5
:10ABA0002ED02A2B38D1154BDB6B95E72D2B30D0CF
:10ABB0002CD32E2B30D1114BDB6C8DE70F4B1B6848
:10ABC0008AE70E4B9B6887E70C4B5B6B84E700BF03
:10ABD000DA93FF1F7886FF1F4096FF1F2896FF1FFE
:10ABE0004896FF1F5496FF1F0C80FF1F5A98FF1FA7
:10ABF0005C98FF1F6D4EC6416C98FF1F9495FF1F18
:10AC00009C4B9B6B68E79B4B1B6C65E7994B5B6CA4
:10AC100062E7984B9B6C5FE7032300E004232370FB
:10AC2000954B1B78002B00F02187944B62681A60CB
:10AC3000934B2AB91A6842F008021A6000F016BF56
:10AC40001A6822F008021A6000F010BFB378022BD5
:10AC50000FD18C4B5B78372B3FF6CFAE8A4903F58B
:10AC6000FF70800001EB83010422FEF75CF800F026
:10AC7000FDBE04233B7000F0F9BEB378022B0ED169
:10AC80007378372B3FF6B9AE7F4903F5FF7080002C
:10AC900001EB83010422FEF782F800F0E7BE0423F3
:10ACA0003B7000F0E3BEB07805283FF684AC754BEE
:10ACB0005B78012B07D002D3022B08D01EE002F0F4
:10ACC000FFF800F0D3BE02F003F900F0CFBE02F0AF
:10ACD00007F9694B78601B78002B00F0C786674B3B
:10ACE0001860674B1A6820B942F008021A6000F039
:10ACF000BDBE22F008021A6000F0B8BE03233B700C
:10AD000000F0B4BEB278022A17D17078072808D8AC
:10AD10001BB9FDF73BFE00F0A9BEFDF723FE00F0D6
:10AD2000A5BEFF2840F0A2865D1C0ABF534BD8B2D7
:10AD30001878FDF73FFE00F099BE04233B7000F049
:10AD400095BEB378012B1CD02BB1022B1FD170788C
:10AD5000FDF75AFE13E07078082802D8FDF73BFE95
:10AD60000DE00A2807D1494B1B6983F40073C3F334
:10AD700040237B600DE0FF280BD1FDF763FE606090
:10AD800007E07078092804D002F044F9F7E70423BB
:10AD90003B70394B1B78002B00F06886374B62689C
:10ADA0001A60374B2AB91A6842F008021A6000F09C
:10ADB0005DBE1A6822F008021A6000F057BE717872
:10ADC0002E4A092925D8DFE801F005080B0E1218D4
:10ADD0001B1E212311680B441AE01168CB1A17E0DF
:10ADE00011684B4314E0116891FBF3F310E0116814
:10ADF00091FBF3F003FB10130AE011680B4007E02E
:10AE000011680B4304E011684B4001E01368DB4319
:10AE1000136012681A4B2AB91A6842F008021A60C5
:10AE200000F024BE1A6822F008021A6000F01EBE6C
:10AE3000124A12689A42124B196804DD21F003018C
:10AE400041F0040108E00BBF21F0060121F00501EB
:10AE500041F0010141F0020119602AB91A6842F07B
:10AE600008021A6000F002BE1A6822F008021A6096
:10AE700000F0FCBD9495FF1F5B98FF1F4C98FF1FCF
:10AE80005096FF1F4896FF1F6C98FF1F80F00F40E1
:10AE900072780C2A00F2EA85DFE802F007111B2520
:10AEA0002F39444E58626C768000B84A12681407F5
:10AEB00040F1DC85B64AC2F8983000F0D7BDB34AFD
:10AEC0001268100700F1D285B14AC2F8983000F03C
:10AED000CDBDAE4A1268D10740F1C885AC4AC2F870
:10AEE000983000F0C3BDA94A1268D20700F1BE85B0
:10AEF000A74AC2F8983000F0B9BDA44A12685707B3
:10AF000040F1B485A24AC2F8983000F0AFBD9F4A24
:10AF1000126812F0050F00F0A9859D4AC2F898301A
:10AF200000F0A4BD994A1268960740F19F85984A9F
:10AF3000C2F8983000F09ABD944A1268950700F064
:10AF40009585934AC2F8983000F090BD8F4A1268F8
:10AF5000D40640F18B858E4AC2F8983000F086BD49
:10AF60008A4A1268900640F18185894AC2F8983071
:10AF700000F07CBD854A1268510640F17785844A0D
:10AF8000C2F8983000F072BD804A1268120640F193
:10AF90006D857F4AC2F8983000F068BD7B4A126820
:10AFA000D70540F163857A4AC2F8983000F05EBD5B
:10AFB000774AC2F8983000F059BD754AD2F89C1013
:10AFC000072900F25385481C02EB8101C2F89C005E
:10AFD000D2F89800C1F8A000C2F8983000F046BD41
:10AFE0006B4BD3F89C20002A00F04085013AC3F84F
:10AFF0009C2003EB8202D2F8A020C3F8982000F036
:10B0000035BD73782E2B04D8624A0121D15400F04B
:10B010002DBDFF2B7FF4F1AC5D4B012283F8C020E6
:10B0200000F024BD73782E2B04D85A4A0021D15445
:10B0300000F01CBDFF2B7FF4E0AC554B002283F8E1
:10B04000C02000F013BD524C94F8C1209AB95E1C88
:10B050004FF00A0205D1504B1B685A43C4F8C42074
:10B0600002E05343C4F8C430FDF7D6FA0123C4F814
:10B07000C80084F8C1306B78042B00F2F784DFE855
:10B0800003F0034C8DC61D00FDF7C6FAD4F8C820A6
:10B09000D4F8C4103E4B801A80EAE072A2EBE07252
:10B0A0008A4204D9002283F8C12000F0DFBCD3F823
:10B0B0009820013AC3F8982000F0D8BCA87801F095
:10B0C0000FFF40B9314B84F8C1001A6822F010021A
:10B0D0001A6000F0CBBCD4F8C4302D4DB3B1FDF7ED
:10B0E0009BFAD5F8C830D5F8C420C01A80EAE073BE
:10B0F000A3EBE073934209D9002385F8C130234BB9
:10B100001A6842F010021A6000F0B0BCD4F898300F
:10B11000013BC4F8983000F0A9BCA878202100F0C9
:10B120000103994041F015014008C9B202F088FAC4
:10B1300010F4007609D0002384F8C130134B1A684C
:10B1400022F010021A6000F091BCD4F8C430104D07
:10B15000ABB1FDF761FAD5F8C830D5F8C420C01AF4
:10B1600080EAE073A3EBE073934208D9074B85F8BC
:10B17000C1601A6842F010021A6000F077BCD4F87F
:10B180009830013BC4F8983000F070BC5096FF1F17
:10B190007886FF1FF895FF1F4C98FF1FA878202185
:10B1A00000F00103994041F015014008C9B202F0D6
:10B1B00047FA10F0010609D0002384F8C130B94BDA
:10B1C0001A6822F010021A6000F050BCD4F8C430A3
:10B1D000B54DABB1FDF720FAD5F8C830D5F8C4208D
:10B1E000C01A80EAE073A3EBE073934208D9AD4B39
:10B1F00085F8C1601A6842F010021A6000F036BC8F
:10B20000D4F89830013BC4F8983000F02FBCA878EF
:10B21000202100F00103994041F015014008C9B216
:10B2200002F00EFA10F0020609D0002384F8C130B3
:10B230009C4B1A6822F010021A6000F017BCD4F878
:10B24000C430994DA3B1FDF7E7F9D5F8C830D5F86A
:10B25000C420C01A80EAE073A3EBE073934207D9DD
:10B26000904B85F8C1601A6842F010021A60FDE345
:10B27000D4F89830013BC4F89830F7E38A4B0022A9
:10B2800083F89420F2E37678142E3FF6B6AB874A23
:10B290009778052F1AD80621854C01FB067144F8D2
:10B2A0002130844B9B7E002B00F0E083002E00F0C9
:10B2B000DD83013E18207043042200F5D36002FBB9
:10B2C000070004EB8101FDF72EFDCFE3FF2F7FF494
:10B2D00072A9774F8EB91825002405F5D060791929
:10B2E0002044214404220434FDF71DFD182CF4D120
:10B2F0001835B5F5FC7FEFD1B8E300246B78182042
:10B300005A1E5043062202FB034100F5D36000EBB6
:10B31000840007EB810104220134FDF704FD062CB3
:10B32000ECD1A3E37378142B3FF667ABB278052A10
:10B3300019D8062101FB03235D4951F823205E4BF8
:10B340007A601B78002B00F091835C4B1A60554BA0
:10B3500022B91A6842F008021A6087E31A6822F0DC
:10B3600008021A6082E3FF2A7FF425A9504E8BB9A8
:10B370001825002405F5D0607119204421440422C9
:10B380000434FDF70CFD182CF4D11835B5F5FC7F0D
:10B39000EFD16BE300246B7818205A1E504306222D
:10B3A00002FB034100F5D36000EB840006EB810152
:10B3B00004220134FDF7F3FC062CECD156E396F899
:10B3C00001803A4FB8F1140F3FF617ABBE78300644
:10B3D00030D50024AB782341D90712D5334B202137
:10B3E0005E7804F00103994041F00101C4F3470085
:10B3F000C9B202F025F9062303FB06462C4B43F89D
:10B4000026002C4B9B7E8BB16B787BB15A1E18208B
:10B4100050432749062202FB034300F5D36000EBAB
:10B42000840001EB83010422FDF77DFC0134062C2E
:10B43000D0D11BE3052E3FF6BEA806F00103202164
:10B44000994041F001017008C9B202F0F9F8194BB6
:10B45000174C9B7E062101FB086644F82600002B52
:10B4600000F004837B78002B00F00083BD78581E29
:10B4700018267043042201FB035100F5D36002FB40
:10B48000050004EB8101FDF74EFCEFE272780B4BF7
:10B490000A2A50D8DFE802F014191F242A32373C58
:10B4A00041464A005096FF1F7886FF1F4896FF1FAF
:10B4B0005496FF1F0C80FF1F5B98FF1F4C98FF1FC7
:10B4C00092491A6809680A4403E090491A680968B1
:10B4D000521A1A602FE08D491A6809684A43F8E742
:10B4E0008A491A68096892FBF1F2F2E7874A1968FB
:10B4F000126891FBF2F002FB1012EAE7834A11682E
:10B500001A680A40E5E7814A11681A680A43E0E7C9
:10B510007E4A11681A684A40DBE77C4A1168C943D1
:10B52000116008E079491A680A6004E0774A1868EF
:10B530001168196010601A68754B22B91A6842F0D8
:10B5400008021A6092E21A6822F008021A608DE27C
:10B55000704B1B68C6F80330FDF7DCFC86E273789D
:10B56000052B00F28382DFE803F003090F151B218E
:10B57000674B1A6802F00F021A6077E2644B1A6890
:10B5800022F010021A6071E2614B1A6822F0200268
:10B590001A606BE25E4B1A6822F040021A6065E2A4
:10B5A0005B4B1A6822F080021A605FE2584B1A68FF
:10B5B00022F480721A6059E272782E2A3FF61DAA90
:10B5C000554901EB8202C2F8CC304FE2524B51494F
:10B5D000D3F888210A604D49D3F88C210A60D3F84A
:10B5E00090214B49C3F89820D3F894210A60D3F8EE
:10B5F000982183F8C120D3F89C21C3F8C820D3F840
:10B60000A021C3F8C420454993F8A421885C08B15F
:10B6100001208854002283F8A82127E2B378052B63
:10B620003EF6C9AF3E4A5278142A3FF6E6A90621F3
:10B6300001FB0233374A3B49126841F8232015E2E7
:10B6400000F006FF12E200F005FF0FE200F003FF3A
:10B650000CE200F001FF09E200F0FFFE06E200F05C
:10B66000FDFE03E22C4B002283F89420FEE1727869
:10B6700012B1012A05D00EE0274B012283F8942055
:10B68000F4E1B3F5C05FBEF496AF234981F894208E
:10B69000C1F89830EAE103233B70E7E11E4B00213B
:10B6A00083F8C01083F8A8111B4A02F1CC034FF0B5
:10B6B000FF3043F8210019480023435401312F295A
:10B6C000F2D182F89430C2F89830C2F89C3082F8F7
:10B6D000C130104A13600D4A13600D4A1360C5E172
:10B6E000127D92070AD4B3F5C05FBEF464AF0A4A74
:10B6F000042182F89410C2F8AC31B7E108233B7002
:10B70000B4E1054B002283F89420AFE16898FF1F55
:10B710005096FF1F4C98FF1F7886FF1FF895FF1F5C
:10B720004896FF1F5496FF1F9849994C92782270B3
:10B730000125B3F5C05F0D7027D2964A127D12EA3B
:10B74000050622D1184602A9FDF740FB9DF80830F6
:10B7500063709DF80930A3709DF80A30E3709DF87E
:10B760000E3023719DF80D3063719DF80C30A3717C
:10B770009DF80B30E37126722B46E15C227A01338F
:10B780000A44082B2272F8D170E101230021E15410
:10B790000133082B7E4AF9D11378137266E173786E
:10B7A000012B1DD00AD3022B2BD1784B01221A700A
:10B7B000784B774A9B781370002319E0734B012272
:10B7C0001A70744B724A9B781370734B186800237D
:10B7D0000133C118082B11F8011CD154F8D145E1EF
:10B7E0001822FA717B7142220523BA713B713DE147
:10B7F0006A4901331944082B11F8091CD154F7D1B7
:10B8000034E103233B7031E17378032B00F22E8186
:10B81000DFE803F0020F1C20614B93F89420FA71CB
:10B8200093F8C120D3F8AC31BA711A0A7A713B711E
:10B830001CE15B4B93F89420FA7193F8C120D3F884
:10B840009830BA711A0A7A713B710FE1554B1B6837
:10B850007B600BE1544B1B687B6007E17278002A28
:10B8600040F00481B178002940F0008140F2D242DA
:10B87000934240F0FB8045F2FF70FDF742FAFDF77E
:10B88000ACFA0120FCF7AAFFF0E07278474B02B156
:10B8900001221A70464BEA781A70414B93F8B011A6
:10B8A000444B1970444900230B7044490B70444BBE
:10B8B00019780A431A70D9E0757815B1012D0FD0A7
:10B8C0001BE0042245F2FB7002A9FDF768FA029B17
:10B8D000D6F803209A4206BF01237B607D60C5E055
:10B8E000B3782A2B06D145F2FB7036490422FDF7C6
:10B8F0001AFABBE003233B70B8E003233B70B5E0CA
:10B900007278032A3ED8DFE802F008022F3A244872
:10B910000022D0F8B411054610E0214AD2F8B41143
:10B92000092907D8481CC2F8B40102EB8102C2F809
:10B93000B8319BE009233B7098E001328A4200F065
:10B940009580214850F822409C424FEA8206F4D16B
:10B950008319481E824204D25C6843F8044B0132CA
:10B96000F7E7C5F8B40181E00D4A0023C2F8B4310D
:10B97000154A002199500433282BF9D176E00A2387
:10B980007B6073E003233B7070E000BF5098FF1FA3
:10B990005198FF1F0C80FF1F0880FF1F00800000D0
:10B9A0007886FF1F4C98FF1F6898FF1FCC93FF1FDE
:10B9B000E193FF1FF795FF1FE093FF1F4696FF1FC0
:10B9C000CD93FF1F4B96FF1F3088FF1F7378812B8D
:10B9D0007EF4F1ADB278274B922A7EF4ECAD9A79E1
:10B9E000A32A7EF4E8AD5A79B42A7EF4E4AD1A793C
:10B9F000C52A7EF4E0ADDB78D62B7EF4DCADFDF716
:10BA0000BAF8FCF709FE0446FCF706FE001B002806
:10BA1000B8BF4042B0F57A7FF6DBFCF7D9FE164B93
:10BA200000221A604FF0FF32C3F87021C3F8702271
:10BA3000C3F87421C3F87422C3F87821C3F87822BC
:10BA4000C3F87C21C3F87C220C4B0D4A1A600120FC
:10BA5000FCF7C4FE0AE040F2D242934206D1094B01
:10BA6000012283F8E02101E00223237004B0BDE845
:10BA7000F08100BF4896FF1F10E000E00080FF1F2C
:10BA8000785634127886FF1F2DE9F843414B424E19
:10BA900000241C60414BC6F898401C60404B86F85F
:10BAA000C1401C6025463F4B03EB85131A7E3E4B7D
:10BAB000A3F1200003F118012AB93C4A32511A516E
:10BAC00002510A5107E03A4A32513A4A1A513A4B66
:10BAD00003513A4B0B5105F001034FF0200808FACF
:10BAE00003F8C5F347095FFA88F848F007014846AC
:10BAF00001F0A6FD324B1851324B0027EF5448F0AD
:10BB00000601484601F09CFD2F4B18512F4BE8B21F
:10BB1000EF54013502F0B7FB062D04F10404C2D145
:10BB20003B462B4A002199500433B3F5806FF8D17E
:10BB3000284FBB7E8BB118250024274905F5D0601E
:10BB400029442044214404220434FDF728F9182C08
:10BB5000F3D11835B5F5FC7FEED1FB7E13B17B7DBB
:10BB60009BB10DE04FF4FF641C49204621440422A0
:10BB7000FDF715F9043440F6D8039C42F4D1EEE702
:10BB8000FCF7A4FF08B1012300E0002386F89430FD
:10BB9000BDE8F8834C98FF1F7886FF1F6898FF1F49
:10BBA0005096FF1FF893FF1FC886FF1F59E2000041
:10BBB0008DE10000F1E10000C9E1000031E2000088
:10BBC0009086FF1FDA93FF1F2896FF1F4096FF1FE6
:10BBD0006C98FF1F0C80FF1F5496FF1F7490FF1F6F
:10BBE000F7B50F4C0F4E86460F4694E80300C6F893
:10BBF00003300D4BB27000228DE803001A7086F8F6
:10BC000000E07770FEF7A0FB084A217882F8E11186
:10BC10009DE80300636884E80300184603B0F0BDA4
:10BC20006098FF1F4896FF1F5B98FF1F7886FF1FD5
:10BC3000F7B51F4E02460C4696E803008DE8030058
:10BC40001C4953780B7093784B70D3788B701379B1
:10BC50008B7153794B7193790B71D379CB70164BF0
:10BC600000271F70FEF770FB144B19786D463346A2
:10BC700071B9217061703278A2707278E270F279D5
:10BC80002271B27962717279A2713279E27109E03E
:10BC9000012907D13A460A4911444978A154013291
:10BCA000082AF8D195E8030083E8030003B0F0BD4B
:10BCB0006098FF1F4896FF1F5B98FF1F5098FF1F5B
:10BCC0005198FF1F014B93F8E10170477886FF1FE1
:10BCD0002DE9F043A84BA94C1B788FB063B1A84B5A
:10BCE0001B78062B08D00A2B06D003F0EF030F2B8E
:10BCF0001CBF002384F8B03194F8B031A14E5A1E15
:10BD0000012A3BD8A049012BCA68079214BF082317
:10BD100007238DF81830327894F8E2318DF8193015
:10BD200000238DF81A30C2B98B688DF82030974BFC
:10BD30008DF8272019788DF8211059788DF8221068
:10BD4000D9798DF8231099798DF8241059791B79B8
:10BD50008DF825108DF8263009E0012A07D101332E
:10BD600006AA8B491A44595CD171082BF7D106A851
:10BD700001F070FA002800F04283A3E0032B1FD1EA
:10BD800033788BB9804F814DB87897F801802A7845
:10BD9000804490446A789044EA799044AA79904427
:10BDA0006A7990442A7918E0012B40F08B800025B5
:10BDB000774B585D0135FCF769FC092DF8D181E01E
:10BDC000042B28D1704F714DB87897F8018000236B
:10BDD00001226B702A706B6080449044FCF756FC23
:10BDE0007878FCF753FC2878FCF750FC6878FCF76F
:10BDF0004DFCE879FCF74AFCA879FCF747FC687928
:10BE0000FCF744FC5FFA88F82879FCF73FFC4046D1
:10BE1000FCF73CFC56E0072B32D133782BBB5A4B56
:10BE200093F802E093F801C0584B8DF800E01F78BA
:10BE30005D78D8798DF80270E644774499798DF869
:10BE400003503D445A798DF8040028441B798DF83D
:10BE5000051001448DF806200A448DF8073013447C
:10BE60008DF801C08DF8083029E0012B27D100237F
:10BE7000474A9A5C0DF803200133092BF8D11EE0E4
:10BE8000082B1FD1414A00230120537010705360CA
:10BE90003D4A8DF80200917852788DF801200A44CD
:10BEA00002448DF800108DF803308DF804308DF8C1
:10BEB00005308DF806308DF807308DF8082068467B
:10BEC000FCF756FE334B1A789846002A00F08B8018
:10BED000314B324D1B78013B062B00F28080DFE8AE
:10BEE00003F00404257E7E7E5F00274A297893684C
:10BEF0008DF8303080238DF831308A238DF8323040
:10BF000000238DF833308DF834308DF835308DF8CE
:10BF100036108DF8293007218DF82A300AA8D36809
:10BF20008DF828100B9301F095F958E0164F2A78F8
:10BF3000B87897F80190814409F10A099144FCF717
:10BF4000A5FB7878FCF7A2FB8020FCF79FFB8A20FA
:10BF5000FCF79CFB0020FCF799FB0020FCF796FB0C
:10BF60000020FCF793FB5FFA89F92878FCF78EFB39
:10BF70004846FCF78BFB32E05A98FF1F7886FF1F7C
:10BF80004896FF1F5098FF1F0C80FF1F6098FF1FEF
:10BF90005198FF1F4696FF1FF795FF1FE093FF1F65
:10BFA000944B2A78987859788DF80D1080230144A5
:10BFB0008DF80E300A318A238DF80C008DF80F3081
:10BFC0008DF8132000230A4403A88DF810308DF853
:10BFD00011308DF812308DF81420FCF7C9FD0023C4
:10BFE0002B7088F80030002384F8B031337094F857
:10BFF000E03113B10120FCF7F1FB06A801F0B6F81F
:10C000000546A0B37C4B9DF820201A709DF8212096
:10C010005A709DF822209A709DF823209A719DF8FD
:10C0200024205A719DF825201A719DF82620DA7077
:10C030009DF8193084F8E231FCF7EEFA6F4B704D41
:10C040001860704B00221A709DF8183094F89420F4
:10C05000072B0CBF0123022385F8B031531E012B9F
:10C06000694B02D9052A40F0A0800022BFE003A856
:10C07000FCF724FB064600285CD0FCF737FB08B130
:10C0800084F8E35194F8E3119DF80C005C4A4B1CD2
:10C09000DBB22144092B84F8E33181F8E40140F05C
:10C0A000BC80002392F8E41182F8E331514A5278BF
:10C0B000914240F0B2801A46514D05F5F271595C3B
:10C0C00001330A44082BD2B2F6D195F8EC319342F1
:10C0D0002CD1494B95F8E5211A7095F8E6215A7054
:10C0E00095F8E7219A7095F8E8219A7195F8E92179
:10C0F0005A7195F8EA211A7195F8EB21DA70FCF77C
:10C100008BFA424B424A186095F894100023137042
:10C11000032285F8B0214A1E012A85F8E3313A4A04
:10C1200002D9052918BF0123137076E0042385F88E
:10C13000B03172E00AAD2846FCF707FD00283BD07D
:10C1400033463246E95C01330A44082BD2B2F9D1B6
:10C150009DF8301091422CD1274B9DF829201A7060
:10C160009DF82A205A709DF82B209A709DF82C205B
:10C170009A719DF82D205A719DF82E201A719DF804
:10C180002F20DA70FCF748FA204B214A1860002370
:10C190001370072284F8B02194F89420511E0129CD
:10C1A0001946194B03D9052A01D001221FE0197045
:10C1B00033E084F8B03130E094F89430104D013B16
:10C1C000012B2AD8D5F89830B3F5C05F22D2FCF7FE
:10C1D0007DFCF8B1D5F898000749431CC5F89830A4
:10C1E000FCF7F4FD092385F8B031074B01221A70E2
:10C1F00013E000BF0C80FF1F4896FF1FE495FF1F50
:10C200007886FF1FB093FF1F5B98FF1FEC95FF1F01
:10C21000F695FF1F002384F8943094F89430794DFC
:10C22000042B04D1784E3278170640F1BD8094F883
:10C23000B03113F0FB0F05D0082B03D0062B01D033
:10C24000FEF782F894F8B031092B40F08480FCF7B7
:10C25000E3F96C4A6D4DD2F888202B68801A80EA89
:10C26000E072A2EBE0729A4209D9694B1A78012A6E
:10C2700004BF02221A70FCF7CFF9C4F88800FCF75B
:10C28000CBF9D4F88C306A68C01A80EAE073A3EB6B
:10C29000E073934209D95E4B5A78012A04BF022207
:10C2A0005A70FCF7B9F9C4F88C00FCF7B5F9D4F86A
:10C2B0009030AA68C01A80EAE073A3EBE07393425F
:10C2C00009D9534B9A78012A04BF02229A70FCF7CD
:10C2D000A3F9C4F8900094F8C030002B3BD0494B30
:10C2E00093F8A821002A36D149498B5C022B2FD123
:10C2F000444B03F1CC0050F82200451C26D04549A0
:10C3000083F8A4210968C3F8881143490968C3F870
:10C310008C11D3F89810C3F890114049C3F89800D5
:10C320000968C3F8941193F8C110C3F8981100225A
:10C33000D3F8C810C3F89C1183F8C120D3F8C410F7
:10C34000C3F8A011012283F8A82104E000238B5434
:10C3500001322F2AC8D194F8B0112A4B092906D1ED
:10C3600093F89420022A04BF052283F89420D4F87D
:10C37000B421244B002A42D0092940D193F89410CB
:10C3800001293CD1D3F8980000231E4901F5DC7443
:10C3900054F82340A04203D1052381F894302EE0C5
:10C3A00001339342F1D12AE095F8B03113F0FB0F3D
:10C3B00025D0082B23D0062B21D0D5F8AC01184C62
:10C3C000D6F803306270B0F5C05F636012D23146B8
:10C3D000FCF7F5FCD5F8AC013146FCF71BFD30B19C
:10C3E000D5F8AC310133C5F8AC31652300E0072343
:10C3F000237004E007232370002385F894300FB0E6
:10C40000BDE8F0837886FF1F4896FF1F9495FF1FB5
:10C41000F895FF1F4C98FF1F6898FF1F5096FF1F4D
:10C420006098FF1F704710B5074CFCF7F5F82368BC
:10C43000C01AB0F5FA7F05D9044B0222DA60FCF786
:10C44000EBF8206010BD00BF6C9CFF1F00F00F4098
:10C450007047704770477047704770477047704724
:10C46000014B53F8200070476888FF1F2DE9F04703
:10C47000B74DEB69B3B1B74B1C781E4694B9FCF7C6
:10C48000CBF8B54B1B68C01AEB690028B8BF404217
:10C49000984207D92046013401F03EFE062CF9D11E
:10C4A000012333702B6AC3B1AC4B1C781D46A4B971
:10C4B000FCF7B2F8AA4BA64A1B68126AC01A80EAB7
:10C4C000E073A3EBE073934207D92046013401F0F7
:10C4D00023FE062CF9D101232B70A24CFCF79CF80B
:10C4E00094F8303004EB83039B69C01A80EAE07350
:10C4F000A3EBE0730A2B2DDDFCF78EF8064694F8CB
:10C500003000202100F00103994041F00101C9B23F
:10C51000400801F095F894F8308004EB8805074650
:10C52000686B381A04F0A4FC8146A869301A04F03C
:10C530009FFC0146484604F0A3FD04F0C9F882A31D
:10C54000D3E9002304F018F904F0B0FB44F8280004
:10C55000AE616F6394F83000824F00F00101202635
:10C5600006FA01F141F015014008C9B201F068F87E
:10C5700010F0400905463CD097F8300000F001016A
:10C5800006FA01F14008C9B201F05AF80138C0B208
:10C5900001280AD997F8300000F0010306FA03F1E8
:10C5A0004008C9B2012201F01BF894F830006E4B2C
:10C5B000012600EA060120271E5407FA01F16B4B01
:10C5C00041F006011E54C9B2F0404FF6FF7201F06F
:10C5D00007F894F8300000EA06018F4047F00701A1
:10C5E0000022F040C9B200F0FBFF94F83030604AFE
:10C5F000D654604B94F830005A4E03EB80129846A4
:10C60000126982B300F00101202707FA01F141F01D
:10C6100002014008C9B201F013F896F8303008EB77
:10C6200083120028B8BF4042126990421BD9F21809
:10C6300092F84C20002A36D14FEA530A03F0010346
:10C640009F4047F01407FFB23946504600F0F8FF0C
:10C65000394640F48062504600F0C2FF96F8303010
:10C660001E4401231DE094F830303E4EE21892F84B
:10C670004C20C2B14FEA530A202703F001039F4028
:10C6800047F01407FFB23946504600F0D9FF39464B
:10C6900020F48062504600F0A3FF96F830301E442C
:10C6A000002386F84C3094F85260DFF8CCA05EB9D5
:10C6B000F0B2FCF790F90AF806000136082EF7D11F
:10C6C000284B012283F8522027260027F8B2FCF7D6
:10C6D00082F91AF8073083421BD0274B07F10C026E
:10C6E000F854264B53F82230022B05D0032B0AD0E6
:10C6F000012B0ED168B106E058B9214A915D01299C
:10C7000007D1935505E01E4B9A5D012A04BF022212
:10C710009A550137082F06F10106D7D194F8303029
:10C7200015F0010104EB03022CD092F85B100029F4
:10C730003DD1012182F85B10104A1A4492F824205E
:10C7400012F0010F29E000BFFCA9F1D24D62904028
:10C750000C80FF1FF695FF1FEC95FF1FB093FF1F86
:10C76000E495FF1F6888FF1FDA93FF1F4096FF1FA5
:10C77000F093FF1FF893FF1FBB88FF1F9495FF1FC7
:10C78000F895FF1F92F85B0088B182F85B10594A58
:10C790001A4492F8242012F0020F08D002211B2222
:10C7A00011FB0323544AD05C012808BFD15494F8EC
:10C7B0003030E218AE0792F861100AD5E9B90121CC
:10C7C00082F861104B4A1A4492F82A2012F0010FA5
:10C7D00009E091B1012182F86110464A1A4492F8A9
:10C7E0002A2012F0020F08D00E33434A12F8131019
:10C7F000012904BF022102F8131015F0800708D0A8
:10C8000094F830303C4A0333D15C012904BF022143
:10C81000D154B9F1000F08D094F83030364A0F33B4
:10C82000D15C012904BF0221D15494F83000334E69
:10C8300008EB80131B6A002B35D06D0533D400F054
:10C840000101202505FA01F141F01901C9B24008A2
:10C8500000F0F6FE804696F8300000F001018D40B1
:10C8600045F001014008C9B200F0EAFE96F8303008
:10C87000234A02EB8312C0EB0800126A80EAE078D8
:10C88000A8EBE07890450ED9184601F045FC96F8E3
:10C8900030301C4A0121D1541533174AD15C01298B
:10C8A00004BF0221D154A7B1174B94F830101A7865
:10C8B00042FA01F0C0070CD50120144D00FA01F135
:10C8C0002970134D28701348007810B922EA01022C
:10C8D0001A7094F83000094D00F05EF894F830308A
:10C8E0000133DBB2052B88BF002385F83030BDE86B
:10C8F000F08700BF9495FF1FF895FF1F6888FF1F02
:10C90000F893FF1FD493FF1FE193FF1FE093FF1FD6
:10C910004696FF1FCC93FF1F2DE9F341DFF874808B
:10C9200018F8003004460E46450800F001076BB1C8
:10C930002021164BB94041F0060153F82420284627
:10C94000C9B200F04DFE002308F80430202303FA9A
:10C9500007F7EDB247F0070186EAE672A2EBE6724E
:10C960002846C9B200F03CFE094A0123002E1355A7
:10C970004FF00002D8BF02230193F9B2009228467B
:10C98000134600F0F1FD02B0BDE8F0812896FF1FCC
:10C99000DA93FF1F4096FF1F2DE9F04F00F00103CF
:10C9A00020269E404508F6B2044646F0150185B0A3
:10C9B000284600F045FEAB4F0246A00107EB000CF5
:10C9C00051089CF80830DCF8049013F0400F02F096
:10C9D000010E09D0385801F0010BC0F1000A5FFACE
:10C9E0008EF1C9F1000905E057F800A05FFA8EFB4F
:10C9F00001F001011F0603F03F0820460391029257
:10CA000008D501F0B1FBD0F1010338BF0023039931
:10CA1000029A06E001F0A8FB029A0399031C18BFD2
:10CA2000012308F1FF30072800F24082DFE810F010
:10CA300008000800080008000201020102010201CA
:10CA4000894F3B5D013B0E2B00F23082DFE813F093
:10CA50000F00230027003300370040004F005E0026
:10CA60009300BA00BF002E02EE0024021E0246F020
:10CA70001401284600F0E4FD07EB84077B4A7A4B5B
:10CA8000B8600121A8F102088845115594BF02221F
:10CA900004221A550AE207EB84039A6808E1002988
:10CAA00000F00482284646F0010100F0C9FD704BF9
:10CAB00043F824001DE107EB84039A6828E1BBF1E9
:10CAC000000F00F0F381204601F026FB0623ECE185
:10CAD00007EB840328469A6846F0140122F003020B
:10CAE00000F07EFD20464946FFF716FF3BE1BBF113
:10CAF000000F40F0DB8120465946FFF70DFF20462E
:10CB0000C9F10001FFF708FF0823CEE1BBF1000FD8
:10CB100000F0CC8146F00101284600F091FD002193
:10CB200080462046FFF7F8FE514B53F82420C8EB0F
:10CB3000020243F8242007EB840328469A6846F053
:10CB4000140122F0030200F04BFD284646F00701D5
:10CB50004A4600F045FD284646F00D01424600F0E9
:10CB60003FFD00221346009201922846314600F014
:10CB7000FBFC092399E1910540F1988146F0010AF7
:10CB80005146284600F05CFD3A4B002118602046D3
:10CB9000FFF7C2FE284646F00D01002200F020FDFE
:10CBA00028465146002200F01BFDA8F10308284644
:10CBB00046F01901002200F013FDB8F1010F00F258
:10CBC0006981FDE0BBF1000F00F0708109E1BBF16C
:10CBD000000F40F06B8146F00101284600F030FD67
:10CBE000594680462046FFF797FE07EB8403284608
:10CBF0009A6846F0140122F0030200F0F1FC284686
:10CC000046F007014A4600F0EBFC0222284646F0B7
:10CC10000D0198FBF2F200F0E3FCCDF800B0CDF886
:10CC200004B0284631465A465B4607E1920540F17A
:10CC30003D812FE10C4F385D01380E2800F236811E
:10CC4000DFE810F01A002E004F005E008000340173
:10CC5000930034013401C500D100AA0000012A016B
:10CC6000240100BFF893FF1FD088FF1FDA93FF1F36
:10CC7000B493FF1F7C95FF1F8E4B0122284646F080
:10CC800014011A5500F0DCFC07EB8403B8F1060F21
:10CC9000986061D0B8F1080F5ED00422864BF8E6A8
:10CCA000B8F1060F0AD107EB84039A6822F0030259
:10CCB000284646F0140142F002020AE0B8F1080FDB
:10CCC00009D107EB840328469A6846F0140122F044
:10CCD000030200F085FC20465146FFF71DFE0323AA
:10CCE000E3E0A8F10502012A05D821B1B8F1060F49
:10CCF00034D10423D9E0002B00F0D8800C23D4E0F9
:10CD0000B8F1050F0AD107EB84039A6822F00302F9
:10CD1000284646F0140142F001020AE0B8F1070F7C
:10CD200009D107EB840328469A6846F0140122F0E3
:10CD3000030200F055FC2046CAF10001FFF7ECFDAC
:10CD40000523B2E0A8F10502012A09D8BBF1000FC2
:10CD500006D0B8F1050F01D10223A6E00F23A4E00D
:10CD6000002B00F0A38007239FE0002B40F09E8063
:10CD7000A8F10708B8F1010F0BD907EB8403284687
:10CD80009A6822F0030246F0140142F0020200F019
:10CD900027FC2046494616E0002B40F08780A8F18A
:10CDA0000708B8F1010F0BD907EB840328469A68EE
:10CDB00022F0030246F0140142F0010200F010FCE0
:10CDC0002046C9F10001FFF7A7FD0A236DE0002B03
:10CDD0006CD0284646F0010100F032FC07EB8403DA
:10CDE00018620B2361E0002B60D146F0010107EBD4
:10CDF00084082846039300F023FCD8F808208246D4
:10CE000046F01401284622F0030200F0E9FB284610
:10CE100046F007014A4600F0E3FBD8F82020924490
:10CE20000222284646F00D019AFBF2F200F0D8FBF0
:10CE3000039B00930193284631461A4600F094FB69
:10CE40000D2332E0930531D50E233B5546F0010703
:10CE50003946284600F0F4FB184B002118602046A4
:10CE6000FFF75AFD284646F00D01002200F0B8FBFE
:10CE700028463946002200F0B3FB284646F0190147
:10CE8000002205B0BDE8F04F00F0AABB204600210B
:10CE9000FFF742FD0E2308E007EB840328469A685B
:10CEA00046F0140100F09CFB00233B5505B0BDE8A3
:10CEB000F08F00BFDA93FF1FD088FF1F7C95FF1F04
:10CEC000024B1A5C0AB901221A547047D088FF1F1E
:10CED000024B1A5C0AB10F221A547047D088FF1F08
:10CEE000014B185C704700BFD088FF1F104A68468E
:10CEF00020F0070113698D4640F273214B434FF632
:10CF0000FF71B3FBF1F36E2B01B504D9094B4FF45C
:10CF10008021596005E04F2B03D8064B4FF4802148
:10CF20009960BDE80140572313608546704700BFF4
:10CF300000B0034080F00F401F4B68461A6820F095
:10CF400007018D4602F01F0201B5072A2DD8DFE840
:10CF500002F0040A2C10161C22281969174A89B2FB
:10CF60001180412222E01969144A89B2518043227A
:10CF70001CE01969114A89B2D180442216E019696E
:10CF80000E4A89B21181452210E019690B4A89B213
:10CF9000518146220AE01969084A89B291814722E3
:10CFA00004E01969054A89B2D1814022BDE80140F7
:10CFB0001A608546704700BF00B00B400889FF1F0C
:10CFC00038B541F23002114B995841F00061995047
:10CFD00041F23C020024995841F00061995003F558
:10CFE000E8230D2540229D604920DC605C621A60C8
:10CFF00001F032FA064B57229D602720DC605C620C
:10D000001A60BDE8384001F027BA00BF0070044044
:10D0100000B003400B2829D8DFE800F006090D1006
:10D02000282828281328191E114B188901E0104BB5
:10D03000588980B270470E4B9889FAE70C4BD88913
:10D04000F7E70B4B588840F2732380B208E0084B97
:10D05000D8888E2380B203E0054B1888422380B223
:10D0600058434FF6FF7390FBF3F070470020704772
:10D070000889FF1F30B541F23C032E4CE55845F0BE
:10D080001005E5502C4B4FF400741C636FF4F875D9
:10D090005C63A3F51433A4F13E542C441C604FF49C
:10D0A00000545C60254C1C601C68E401FCD5013810
:10D0B000072813D8DFE800F0100E0C0A0812060447
:10D0C0001F480CE01F480AE01F4808E01F4806E020
:10D0D0001F4804E01F4802E01F4800E01F48586056
:10D0E0001F4B002058631F4818601F488D044FF0E5
:10D0F00080642840C3F88040C3F884003AB11A48DD
:10D10000C3F8904094042040C3F8940001E0C3F8B1
:10D1100090204FF08464C3F8A0401148C3F8A410D5
:10D1200022B1C0F8B040C0F8B42030BDC0F8B02083
:10D1300030BD00BF00700440009004400F008050DC
:10D140008720FE018720FE038720FE0F8720FE1325
:10D150008720FE278720FE638720FEC78720FE07E3
:10D16000004002400F0080000000FC1F384BD3F845
:10D170008020C2F30362022A10B513D0D3F89020A6
:10D18000C2F30362022A0FD0D3F8A020C2F30362D5
:10D19000022A0AD0D3F8B030C3F30363022B54D170
:10D1A000032202E0002200E00122120102F14023EA
:10D1B00003F50033D3F88010C1F303410170D3F8B5
:10D1C000801011F4801118BF01218170D3F88010F4
:10D1D00011F4001118BF01214170417821B9D3F831
:10D1E0008410C1F38A4103E0D3F8841021F0604138
:10D1F00002F1402202F500324160D2F88840240E4C
:10D200000472D2F88840240C4472D2F88840240A70
:10D21000847202F18801D2F88820C2724A68120E24
:10D2200002734A68120C42734A68120A82734A688F
:10D23000C273D3F8802092024CBF4FF084624FF04B
:10D240008062C3F88020012010BD002010BD00BF07
:10D2500000400240204BD3F87021C2F303620C2A35
:10D2600038D04178426811B1C2F3110202E0910452
:10D270001A4A0A40C3F87421427A037A120442EA35
:10D280000362C37A1A43837A42EA0322124BC3F839
:10D290007821427B017B120442EA0162C17B0A438E
:10D2A000817B42EA0122C3F87C2143788278002BFB
:10D2B00014BF4FF042634FF040630AB143F4801350
:10D2C0000278120402F470221343034A0120C2F8C8
:10D2D0007031704700207047004002400000FC1F82
:10D2E0000B4B4FF00062C3F870214FF48022C3F85B
:10D2F0007421084AC3F878216FF48471A2F1663270
:10D300000A44C3F87C21044AC3F87021704700BF67
:10D3100000400240785634120000080C684620F0A5
:10D3200007018D4611B53D4BDA7842F00202DA7002
:10D330003B4A1078C0B20228114641D0032835D0AC
:10D34000012867D1547891788C4216D2D978C907D0
:10D3500009D451785068C9B24C1CE4B25470425C94
:10D36000D2B21A7156E0997801F0DF01997099787C
:10D3700001F0EF01997010724AE0517A01F0FF005C
:10D3800049B9997801F0DF019970997801F0EF01BE
:10D39000997010703EE0997841F004019970917A8B
:10D3A000C9B2197100235372032332E0997801F056
:10D3B000EF0199701B79D168DBB20B70022328E072
:10D3C000147C507C84421FD2507C127C821A012A29
:10D3D00005D19A7802F0DF029A7000230B704A7C24
:10D3E0000B7CD31A022B04DC0C4B9A7842F0080217
:10D3F0009A700B7CCA68DBB2581CC0B2087407492B
:10D400000979C9B2D15405E0997801F0DF0199702A
:10D4100000231370BDE81140854670470070064038
:10D420001889FF1F0B4A41F234031920D15841F0EB
:10D430008001D150084B4FF400729A62DA6203F512
:10D44000E0331B225A70C0229A7000225A7101F0F8
:10D4500003B800BF0070044000B0044010B5124B88
:10D460000024D2B21C725C729A7001225C701A7035
:10D470000E4A5960917801F0F7019170917841F06E
:10D4800010019170917800F0FE0041F02001917040
:10D4900010711A78002AFCD1034B187AD0F10100E0
:10D4A00038BF002010BD00BF1889FF1F0070064064
:10D4B00010B5124B0024D2B21C725C725A74032253
:10D4C0001C741A700E4AD960917801F0F7019170BE
:10D4D000917841F010019170917840F0010041F095
:10D4E0002001917010711A78002AFCD1034B187A30
:10D4F000D0F1010038BF002010BD00BF1889FF1F08
:10D500000070064070B5164C0025E36001269DF8BA
:10D5100010302572D2B26672A2706570637440EAF0
:10D5200006032574A3720F4B616026709A7802F08F
:10D53000F7029A709A7842F010029A709A7800F086
:10D54000FE0042F020029A7018712378002BFCD163
:10D55000034B187AD0F1010038BF002070BD00BF26
:10D560001889FF1F007006402DE9F0471F461A4B2F
:10D570009DF8206033F810409DF824509046814675
:10D580008A46002241F080012046FBF749FB4146D4
:10D5900000222046FBF744FB394600222046FBF7D9
:10D5A0003FFB0AF07F0A314600222046FBF738FB9A
:10D5B00047EA08272946204601220AEB4A0AFBF7D8
:10D5C0002FFB46EA0726D144044B45EA062543F8DB
:10D5D0002950BDE8F08700BF981701002C89FF1F74
:10D5E000F8B5154B33F81050144606460F46002286
:10D5F00041F080012846FBF713FB210E002228464C
:10D60000FBF70EFBC4F3074100222846FBF708FB9B
:10D6100007F07F07C4F3072100222846FBF700FB31
:10D6200007EB47072846E1B20122FBF7F9FA3E442F
:10D63000024B43F82640F8BD981701002C89FF1FC4
:10D64000294B70B501F07F055A19127B002A43D08F
:10D6500033F81040294600222046FBF7E1FA00216A
:10D660000A462046FBF7DCFA00210A462046FBF773
:10D67000D7FA00210A462046FBF7D2FA0021012200
:10D680002046FBF7CDFA00210A462046FBF7C8FAF0
:10D6900000210A462046FBF7C3FA002106020A468B
:10D6A0002046FBF7BDFA0021304306020A46204619
:10D6B000FBF7B6FA30430602002120460122FBF7B1
:10D6C000AFFA222D46EA000001D0422D0AD1030212
:10D6D00008D540F07F4070BD05EB45052844034B5D
:10D6E00053F8200070BD00BF981701002C89FF1F60
:10D6F000F8B50E4C04440D4694F800269AB900F093
:10D700000106360146F06C064708F6B23146384647
:10D71000FFF796FF05F00F0320F00F023146384661
:10D720001A43FFF75DFF84F80656F8BD2C89FF1FEA
:10D7300070B500F00104240144F06C044508E4B223
:10D740000E4628462146FFF77BFF06F0070220F031
:10D7500070032146284643EA0212BDE87040FFF7F5
:10D760003FBF70B500F00104240144F06C0445088B
:10D77000E4B20E4628462146FFF762FF06F00F028C
:10D7800020F4F0632146284643EAC212BDE8704007
:10D79000FFF726BF70B500F00104240144F06C04CB
:10D7A0004508E4B20E4628462146FFF749FF06F039
:10D7B000030220F4C0332146284643EAC232BDE8C2
:10D7C0007040FFF70DBF70B500F00104240144F074
:10D7D0006C044508E4B20E4628462146FFF730FFA8
:10D7E00006F00F0220F470032146284643EA025255
:10D7F000BDE87040FFF7F4BE70B500F001042401ED
:10D8000044F06C044508E4B20E4628462146FFF772
:10D8100017FF06F00F0220F070632146284643EA06
:10D820000262BDE87040FFF7DBBE70B500F0010496
:10D83000240144F06C044508E4B20E462846214613
:10D84000FFF7FEFE16B140F0804201E020F080427A
:10D8500028462146BDE87040FFF7C2BE70B500F013
:10D860000104240144F06C044508E4B20E46284645
:10D870002146FFF7E5FE16B140F4002201E020F456
:10D88000002228462146BDE87040FFF7A9BE70B5CA
:10D8900000F00104240144F06C044508E4B20E4693
:10D8A00028462146FFF7CCFE16B140F4802201E065
:10D8B00020F4802228462146BDE87040FFF790BE44
:10D8C00070B500F00104240144F06C044508E4B292
:10D8D0000E4628462146FFF7B3FE16B140F48042BB
:10D8E00001E020F4804228462146BDE87040FFF761
:10D8F00077BE70B500F00104240144F06C044508C3
:10D90000E4B20E4628462146FFF79AFE16B140F4CF
:10D91000005201E020F4005228462146BDE8704044
:10D92000FFF75EBE70B500F00104240144F06C0402
:10D930004508E4B20E4628462146FFF781FE16B19F
:10D9400040F4805201E020F4805228462146BDE890
:10D950007040FFF745BE70B500F00104240144F0AB
:10D960006C044508E4B20E4628462146FFF768FEDF
:10D9700033074CBF20F0700320F4076306F0070262
:10D9800048BF43F400632846214643EA0212BDE83B
:10D990007040FFF725BE70B500F00104240144F08B
:10D9A0006C044508E4B20E4628462146FFF748FEBF
:10D9B00006F00F0220F4F0632146284643EAC21223
:10D9C000BDE87040FFF70CBE70B500F00104240103
:10D9D00044F06C044508E4B20E4628462146FFF7A1
:10D9E0002FFE16B140F4003201E020F40032284648
:10D9F0002146BDE87040FFF7F3BD08B5094B03446D
:10DA000093F8002652B900F00101090141F06C01C0
:10DA10004008FFF715FE00F00F0008BD93F806065A
:10DA200008BD00BF2C89FF1F00F00101090108B5E6
:10DA300041F06C01C9B24008FFF702FEC0F30210CA
:10DA400008BD00F00101090108B541F06C01C9B23F
:10DA50004008FFF7F5FDC0F3C31008BD00F0010159
:10DA6000090108B541F06C01C9B24008FFF7E8FDB3
:10DA7000C0F3C13008BD00F00101090108B541F053
:10DA80006C01C9B24008FFF7DBFDC0F3035008BDCD
:10DA900000F00101090108B541F06C01C9B240086C
:10DAA000FFF7CEFDC0F3036008BD00F001010901DE
:10DAB00008B541F06C01C9B24008FFF7C1FDC0F3E1
:10DAC000807008BD00F00101090108B541F06C014A
:10DAD000C9B24008FFF7B4FDC0F3C04008BD00F074
:10DAE0000101090108B541F06C01C9B24008FFF716
:10DAF000A7FDC0F3804008BD00F00101090108B591
:10DB000041F06C01C9B24008FFF79AFDC0F38030C4
:10DB100008BD00F00101090108B541F06C01C9B26E
:10DB20004008FFF78DFDC0F3403008BD00F0010153
:10DB3000090108B541F06C01C9B24008FFF780FD4A
:10DB4000C0F3003008BD00F00101090141F06C0193
:10DB500008B5C9B24008FFF773FDC0F30213020510
:10DB600048BF43F00803184608BD00F00101090151
:10DB700008B541F06C01C9B24008FFF761FDC0F380
:10DB8000C31008BD00F00101090108B541F06C01A6
:10DB9000C9B24008FFF754FDC0F3404008BD70B55E
:10DBA00000F00104240144F06D044508E4B20E467F
:10DBB00028462146FFF744FD06F0030220F06003EB
:10DBC0002146284643EA4212BDE87040FFF708BDEF
:10DBD00070B500F00104240144F06D044508E4B27E
:10DBE0000E4628462146FFF72BFD06F0030220F4DF
:10DBF000C0432146284643EA4232BDE87040FFF761
:10DC0000EFBC70B500F00104240144F06D04450838
:10DC1000E4B20E4628462146FFF712FD06F00F0239
:10DC200020F470632146284643EA0222BDE8704092
:10DC3000FFF7D6BC70B500F00104240144F06D0478
:10DC40004508E4B20E4628462146FFF7F9FC06F0E7
:10DC50000F0320F00F02214628461A43BDE870400A
:10DC6000FFF7BEBC70B500F00104240144F06D0460
:10DC70004508E4B20E4628462146FFF7E1FC20F4B1
:10DC80007F022146284642EA0642BDE87040FFF77F
:10DC9000A7BC70B500F00104240144F06D044508F0
:10DCA000E4B20E4628462146FFF7CAFC16B140F4FE
:10DCB000004201E020F4004228462146BDE87040C1
:10DCC000FFF78EBC70B500F00104240144F06D0430
:10DCD0004508E4B20E4628462146FFF7B1FC16B1CE
:10DCE00040F0807201E020F0807228462146BDE8B5
:10DCF0007040FFF775BC00F00101090108B541F063
:10DD00006D01C9B24008FFF79BFCC0F3411008BD8C
:10DD100000F00101090108B541F06D01C9B24008E8
:10DD2000FFF78EFCC0F3413008BD00F0010109018E
:10DD300008B541F06D01C9B24008FFF781FCC0F39E
:10DD4000032008BD00F00101090108B541F06D0193
:10DD5000C9B24008FFF774FC00F00F0008BD00F0E6
:10DD60000101090141F06D0108B5C9B24008FFF792
:10DD700067FC0314D8B21B0648BF60F0FF0008BD63
:10DD800000F00101090108B541F06D01C9B2400878
:10DD9000FFF756FCC0F3C03008BD00F001010901D7
:10DDA00008B541F06D01C9B24008FFF749FCC0F366
:10DDB000006008BDF8B510F001064FEA50040F46A8
:10DDC00020460CBF10211821FFF73AFC07F0030290
:10DDD00020F44015002E204645EA02520CBF1021C7
:10DDE0001821BDE8F840FFF7FBBB70B510F0010645
:10DDF0004FEA50040D4620460CBF10211821FFF7B2
:10DE00001FFC15B140F4802201E020F48022002E96
:10DE100020460CBF10211821BDE87040FFF7E0BB81
:10DE2000F8B510F001064FEA50040F4620460CBF2B
:10DE300010211821FFF704FC07F0030220F44035FD
:10DE4000002E204645EA02420CBF10211821BDE8F1
:10DE5000F840FFF7C5BB70B510F001064FEA50045B
:10DE60000D4620460CBF10211821FFF7E9FB002EBC
:10DE700020F47F4242EA052220460CBF10211821DF
:10DE8000BDE87040FFF7ACBB70B510F001064FEA7B
:10DE900050040D4620460CBF10211821FFF7D0FB7F
:10DEA000002E20F0FF0242EA050220460CBF10219E
:10DEB0001821BDE87040FFF793BB10F0010F08B5C3
:10DEC0000CBF102118214008FFF7BAFBC0F3015026
:10DED00008BD10F0010F08B50CBF10211821400833
:10DEE000FFF7AEFBC0F3804008BD10F0010F08B58E
:10DEF0000CBF102118214008FFF7A2FBC0F301401E
:10DF000008BD10F0010F08B50CBF10211821400802
:10DF1000FFF796FBC0F3072008BD10F0010F08B50E
:10DF20000CBF102118214008FFF78AFBC0B208BDC2
:10DF300010F0010F08B514BF192111214008FFF797
:10DF40007FFBC0B208BD2DE9F743FAF765FB044635
:10DF5000FAF762FB001B0028B8BF40420928F7DD32
:10DF60000027FCB201264FF03509002520466C2120
:10DF7000002233464FF014088DE84002FFF7F4FA10
:10DF8000204630212A460723CDF800800195FFF76F
:10DF9000EBFA20467C212A4633468DE84002FFF703
:10DFA000E3FA0723204650212A46CDF80080019548
:10DFB000FFF7DAFA204629462A46FFF711FB2046EA
:10DFC00020212A46FFF70CFB20462D212A46FFF789
:10DFD00007FB204621212A46FFF702FB204640216D
:10DFE0002A46FFF7FDFA20464D212A46FFF7F8FAA8
:10DFF000204641212A46FFF7F3FA204623213246E4
:10E00000FFF7EEFA20462421DC22FFF7E9FA20464A
:10E01000252146F6DB02FFF7E3FA2046262140F2EF
:10E02000B712FFF7DDFA204627214DF2B712FFF7AE
:10E03000D7FA2046282140F2B712FFF7D1FA20463E
:10E040002A21DC22FFF7CCFA20462B210A22FFF7F7
:10E05000C7FA204643213246FFF7C2FA2046442140
:10E06000DC22FFF7BDFA2046452146F6DB02FFF72A
:10E07000B7FA2046462140F2B712FFF7B1FA204620
:10E0800047214DF2B712FFF7ABFA2046482140F284
:10E09000B712FFF7A5FA20464A21DC22FFF7A0FAC3
:10E0A000374420464B210A22FFF79AFA032F7FF4C8
:10E0B00058AFE8B2FFF7A1FC054B5855063B0022CC
:10E0C000EA540135062DF4D103B0BDE8F08300BF5A
:10E0D000328FFF1F38B5074C044494F8001641B93D
:10E0E00094F80656FFF704FB012384F8003684F801
:10E0F000065638BD2C89FF1F064B034493F80026B3
:10E1000032B1002293F8061683F80026FFF7F0BA22
:10E11000704700BF2C89FF1F73B5114B012600EA21
:10E12000060120241E548C400E4BC0F34705E4B278
:10E130001E5444F0070128460022FFF751FA2846F2
:10E1400044F006014FF6FF72FFF74AFA00228DE80D
:10E150004400284621461346FFF706FA02B070BD78
:10E16000DA93FF1F4096FF1F10F0010F08B54FF024
:10E1700004014FEA500004D0FFF762FAC0F34010E8
:10E1800008BDFFF75DFAC0F3001008BD002808B510
:10E1900009DB02F08BFA0AA3D3E9002302F016FC94
:10E1A00003F032FA08E002F081FA05A3D3E9002374
:10E1B00002F00CFC03F098F902F078FD08BD00BFF6
:10E1C00034F7FFFF7F84EE3F08B502F06FFA06A335
:10E1D000D3E9002302F0FAFB03F016FA02F066FD21
:10E1E00008BD00BFAFF30080EB1100A2941A5D40A0
:10E1F000002808B509DB02F059FA0BA3D3E9002384
:10E2000002F0BAFA03F070F908E002F04FFA06A340
:10E21000D3E9002302F0B0FA03F0F6F902F046FD6C
:10E2200008BD00BFAFF3008034F7FFFF7F84EE3FEF
:10E2300008B502F03BFA06A3D3E9002302F09CFAEA
:10E2400003F052F902F032FD08BD00BFAFF30080C9
:10E25000EB1100A2941A5D40704700BFAFF300803D
:10E2600010B50024E0B200F001032021994041F0F4
:10E270001A014008C9B24FF480320134FFF7B0F9F7
:10E28000062CEFD110BD2DE9F347594C04EB801457
:10E29000183463684FEA500900F001080BB1658833
:10E2A000C5B9202303FA08F85FFA88F85FFA89F9FC
:10E2B00048F0180421464846FFF7C2F9214620F4E9
:10E2C00080624846FFF78CF9484648F01A014FF43F
:10E2D000803282E0FFF7DCFBC0F1080005FA00F0B5
:10E2E00002F0E4F9D4F804A004468AEAEA70A0EB4C
:10E2F000EA700D4602F0DAF902460B46204629463E
:10E3000002F064FB3B4B002204460D4602F034FA57
:10E310006A4606460F4603F017F80022002302F073
:10E3200093FCC0B13946304602F0C0FC202303FA0A
:10E3300008F85FFA88F8BAF1000F5FFA89F948F037
:10E34000180504462946B8BF44424846FFF778F905
:10E3500020F4806239E0204629466A4602F0F4FF44
:10E36000BAF1000F04460D46DDE900010CDD02F0B4
:10E370009DFC1DA3D3E9002306042946204602F094
:10E38000FBF902F093FC0FE002F090FCC04316A3EF
:10E39000D3E9002306042946204602F0EDF902F0F5
:10E3A00085FCC0F51C501030202303FA08F85FFAF2
:10E3B00088F85FFA89F948F0180540EA060429460A
:10E3C0004846FFF73DF940F4806248462946FFF78A
:10E3D00007F9484648F01A01224602B0BDE8F04766
:10E3E000FFF7FEB8AFF30080000000000088C340D4
:10E3F000F893FF1F0000F04000F001032021994036
:10E4000041F019014008C9B2FFF71AB900F0010341
:10E410000A462021994041F019014008C9B2FFF78E
:10E42000DFB800BFAFF30080FEE74FF0E023084AFB
:10E43000C3F8082D074A4CF22053D3814DF6281318
:10E44000D381138823F001031B041B0C1380704736
:10E450000080000000200540802810B54FF0010129
:10E46000154A06DD00F01F008140C2F88C11D16012
:10E4700010BD402806DD00F01F008140C2F8881161
:10E48000916010BD20280C4606DD00F01F00814081
:10E49000C2F88411516010BD084B0340002B03DA11
:10E4A000013B63F01F030133034A04FA03F3C2F88C
:10E4B0008031136010BD00BF00E100E01F0000804C
:10E4C000802810B54FF00102134905DD00F01F0050
:10E4D0008240C1F88C2010BD402805DD00F01F00EF
:10E4E0008240C1F8882010BD2028144605DD00F0C8
:10E4F0001F008240C1F8842010BD084B0340002B50
:10E5000003DA013B63F01F030133034A04FA03F308
:10E51000C2F8803010BD00BF00E100E01F000080A5
:10E5200003291ADC202818DC04220C4B90FBF2F2A1
:10E53000D2B2034002F160428901002B02F564422D
:10E54000C9B203DA013B63F003030133DBB21068A5
:10E55000DB0001FA03F318431060704703000080EA
:10E56000064B1A78D2B2012A05D1222902D02129DC
:10E5700001D100225A7001225A707047388FFF1F54
:10E5800070B5144611B91B4B197070BD022903D127
:10E59000184B01221A7070BD042914D1154B5B78F9
:10E5A000012B25D195880023402D28BF40255E1CD6
:10E5B000DBB2AB4205D22268D05C00F0C7F833462C
:10E5C000F5E7002007E003290CD10A4B5A78012A0D
:10E5D0000ED100209870022102460346BDE870402B
:10E5E00000F046BF052903D1024B00221A705A7071
:10E5F00070BD00BF388FFF1F10B50446204600F0E5
:10E60000BDF80028FAD110BD704710B5084C02467D
:10E610000B4600200121A17000F0EEFA224618B14D
:10E620000023A370122010BD9378002BFCD110BDE5
:10E63000388FFF1FF8B506460F4600F0FAFC0E4B68
:10E640001A78012A16D15B78012B13D100F000F95A
:10E6500088B10025ECB2BC4205D330462146BDE866
:10E66000F840FFF7D2BF301900F0D6F80135002886
:10E67000F0D0F2E70C20F8BD388FFF1F08B540211D
:10E680000248FFF7D7FF00F095F808BD3B8FFF1F4A
:10E6900038B5054600F0A8F80B28044609D106480D
:10E6A0004021FFF7C7FF28B92846BDE8384000F0F1
:10E6B0009BB80024204638BD7B8FFF1FF8B500248F
:10E6C00006460F462546A3B29F4207D0305DFFF7AE
:10E6D000DFFF002818BF0B250134F4E72846F8BDFA
:10E6E00038B5451E002415F8010F28B1FFF7D0FFFB
:10E6F000002818BF0B24F6E7204638BD07B50123D4
:10E70000002000930549064B024600F01FFA00283E
:10E7100014BF1B20002003B05DF804FB81E500005E
:10E7200061E5000038B50D46044600F097F88542D3
:10E730000AD825440020AC4207D020B914F8010BB8
:10E7400000F052F8F7E738BD0B2038BD10B50A4B82
:10E75000197840290ED05A789C180132D2B2402A3A
:10E76000A07001F101014FF00000197014BF5A7040
:10E77000587010BD0B2010BDBB8FFF1F10B50C4B88
:10E78000197891B193F842209C180132D2B2A47842
:10E790000470402A4FF0000001F1FF31197014BFDE
:10E7A00083F8422083F8420010BD0A2010BD00BF4C
:10E7B000BB8FFF1F014B1878704700BFBB8FFF1F37
:10E7C000024B1878C0F14000C0B27047BB8FFF1FEA
:10E7D000034B00225A7083F842201A70704700BF22
:10E7E000BB8FFF1FFFF7F4BF10B50A4B1978402904
:10E7F0000ED05A789C180132D2B2402AA07001F192
:10E8000001014FF00000197014BF5A70587010BD0C
:10E810000B2010BDFE8FFF1F10B50C4B197891B166
:10E8200093F842209C180132D2B2A4780470402A96
:10E830004FF0000001F1FF31197014BF83F842203E
:10E8400083F8420010BD0A2010BD00BFFE8FFF1FDD
:10E85000014B1878704700BFFE8FFF1F024B1878DE
:10E86000C0F14000C0B27047FE8FFF1F034B002273
:10E870005A7083F842201A70704700BFFE8FFF1F46
:10E88000FFF7F4BF70B50446007801F08DF9017808
:10E890000023DAB28A4208D203EB83050544667886
:10E8A0006D78AE4203F10103F3D1154D207A342384
:10E8B00003FB0253D97810B998780130987034234B
:10E8C0005A43AB189B788B420DD003F003030C2105
:10E8D00001FB03220A4B1A44131D107951791B893D
:10E8E000926800F091FBD5F89C3043B1227A002A5F
:10E8F000224614BF0521032112F8080B984770BD6A
:10E900004490FF1F2DE9FF470D4691468DF80F00FB
:10E9100001F04AF9022D064649D190F800A00024E2
:10E92000E3B2534504F1010409DA03EB83033344F2
:10E930000DF10F005978DA7801F0F6F9F0E74FF0B1
:10E9400000085FFA88F7574527DA07EB870737444F
:10E950007C1C6078A3787978B4F8032000900020BC
:10E9600001900DF10F0001F0BDF96378032B05D183
:10E970009DF80F007978184A01F03CFA7978A3786D
:10E9800041F0100141EAC3110DF10F00C9B200229C
:10E9900001F0FAF908F10108D3E7104BD3F89C30E5
:10E9A000B3B19DF80F0029464A46984710E0002D64
:10E9B000F3D12B463278591CDBB29A42EDD9074A83
:10E9C000342000FB032300229A70DA700B46F1E733
:10E9D00004B0BDE8F08700BF85E800004490FF1F49
:10E9E0002DE9F0410C7804F06004202C1D4638D14C
:10E9F0004C78042C1CD00AD8012C2ED02DD3022CFC
:10EA00001FD0032C29D1BDE8F04100F05FB9212CC3
:10EA10001BD005D8202C20D1BDE8F04100F03EB934
:10EA2000222C16D0232C18D1BDE8F04100F046B9B5
:10EA300002241C801468002525701468671C176068
:10EA40006570BDE8F04100F05BB9BDE8F04100F051
:10EA50001DB9BDE8F04100F07BB900202880BDE879
:10EA6000F081402C06D1054CD4F8A04014B1A04749
:10EA7000BDE8F081CD20BDE8F08100BF4490FF1FCC
:10EA800073B50446007801F08FF863680093A27AAA
:10EA9000637A43EA0223ADF8043001780023DAB246
:10EAA0008A4208D203EB8305054466786D78AE424E
:10EAB00003F10103F3D1164D207A342303FB0253F3
:10EAC000D97810B998780130987034235A43AB182C
:10EAD0009B788B420DD003F003030C2101FB032232
:10EAE0000B4B1A44131D107951791B89926800F061
:10EAF0008BFAD5F89C304BB1227A20781AB10521D7
:10EB000004F1080201E003216A46984702B070BD93
:10EB10004490FF1F07B543680093437A817A43EA24
:10EB20000123ADF80430084BD3F89C30024643B1C2
:10EB3000017A007811B10521083201E004216A460A
:10EB4000984703B05DF804FB4490FF1F2DE9F8439C
:10EB5000054688461746994601F026F802789DF842
:10EB600020300132064600212846D2B201F09CF83E
:10EB7000044630BB28461449144A00F08EF9337815
:10EB8000601CE4B2A34211D904EB84023244342362
:10EB90005C430F4992F801E001F804E00B19927808
:10EBA0005A7000229A70DA700446E8E7284649460F
:10EBB00000F066F8044620B9054BC3F89C80C3F802
:10EBC000A0702046BDE8F88305E90000E1E90000F7
:10EBD0004490FF1F08B5074B0022C3F89C20C3F8E0
:10EBE000A02000F0ADF918B9BDE8084001F072B8F6
:10EBF00008BD00BF4490FF1F2DE9F047914607462E
:10EC00000D46984600F0D0FF02780024E3B293420C
:10EC100007D2013404EB8401014411F8041CA94219
:10EC2000F4D1164A342058431118CE788B78F41A50
:10EC3000E4B2042C02D1C120BDE8F08706F0030441
:10EC40004FF00C0C0CFB040414440136F6B227718F
:10EC50006571C4F80890A4F80C80CE70F61AF6B26C
:10EC6000012E07D1384629464A464346BDE8F047BB
:10EC700000F0CAB90020BDE8F08700BF4490FF1F34
:10EC8000014B002019607047E890FF1F024B097983
:10EC9000197100F08DBF00BFE890FF1F13B500246D
:10ECA00002AA1C80044B42F8041D0979197100F076
:10ECB0008DFF02B010BD00BFE890FF1F002018803C
:10ECC000014B4A88DA807047E890FF1F30B50C4648
:10ECD0000221198021796488084D012C297103D102
:10ECE000BDE8304000F08ABF022C03D1BDE83040BF
:10ECF00000F090BF0020188030BD00BFE890FF1FDB
:10ED000030B50C460221198021796488084D012C08
:10ED1000297103D1BDE8304000F088BF022C03D137
:10ED2000BDE8304000F094BF0020188030BD00BF27
:10ED3000E890FF1F044B054A19791B7A1171137271
:10ED400003210A23FFF758BFE890FF1F4C80FF1FE5
:10ED500070B500261E808B780E4CC3F340014A002C
:10ED6000637261F3000203F00103A372054622728D
:10ED7000FFF7E0FF23685BB1617A01F0020101F067
:10ED8000FF02284611B12221324600E02121984796
:10ED9000002070BDE890FF1F08B50246034B12F833
:10EDA000080B1B680521984708BD00BFF490FF1FA2
:10EDB00038B5084D04462A1D012100F0CDFF20463C
:10EDC0000121802200F0E0FF2B6820780A21002238
:10EDD000984738BDF490FF1F37B501210DF10702A8
:10EDE000044600F0B9FF9DF80730074D802B04D191
:10EDF000204601212A7900F0C7FF2B6820780B21DB
:10EE00000022984703B030BDF490FF1F43680521EE
:10EE10005A7800F0B9BF73B50122002405460126D7
:10EE2000002100F081FF334621468DE8500028463E
:10EE3000102200F057FF21462246284600F074FFBA
:10EE4000234621468DE850002846102200F04AFF54
:10EE500031462846022200F097FF32462846062116
:10EE600000F092FF22462846902100F08DFF044BCF
:10EE700028781B6821462246984702B070BD00BF23
:10EE8000F490FF1F42783AB9C178C90141F01001EE
:10EE900001F0900100F078BF704773B50C468DF813
:10EEA000070001F0FBF91F4E34600446002836D1FC
:10EEB00010211D4A9DF8070000F09CFF1221044616
:10EEC0001A4A9DF8070000F095FF2043C4B21421B0
:10EED000174A9DF8070000F08DFF2043C4B21321AC
:10EEE000144A9DF8070000F085FF2043C4B21721A3
:10EEF000114A9DF8070000F07DFF02AD2043C4B227
:10EF0000162115F8010D0D4A00F074FF2043C4B21C
:10EF100001212846032200F037FF032333712046E6
:10EF200002B070BDF490FF1F17EE00000DEE000060
:10EF3000B1ED0000D9ED000085EE000099ED000074
:10EF400037B502AC174B04F8010D00221021204602
:10EF50001A6000F051FF12210546204600F04CFFD8
:10EF60002843C5B21421204600F046FF2843C5B20D
:10EF70001321204600F040FF2843C5B21721204648
:10EF800000F03AFF2843C5B21621204600F034FFB6
:10EF9000284310F0FF0003D19DF8070001F08AF923
:10EFA00003B030BDF490FF1F30B585B004AC012133
:10EFB00004F8090D0DF10E02204600F0CDFE2046AA
:10EFC00006210DF10F0200F0C7FE9DF80E30802BD8
:10EFD00016D19DF80F309B0712D59DF8070000F061
:10EFE000E1FD012805460BD172B6204600F038FB42
:10EFF0000022204629468DF80E2000F0C5FE62B69C
:10F000009DF80E0005B030BD73B50E4615461C4682
:10F010008DF80700FFF7C8FF802807D00DF1070023
:10F0200031462A46234600F0B9FA00E0002002B03B
:10F0300070BD7047062812D880000129C0B204BFF5
:10F040000230C0B2074AC0F34703122101FB032379
:10F050001A884FF6FF739A4208BFFF207047FF20BF
:10F06000704700BFFC90FF1F2DE9F041334D344C39
:10F07000344E002785F800714FF4107284F8400276
:10F0800088462046FF2102F015F9304639464FF4F4
:10F090008062C4F8446202F00DF995F80C3143F037
:10F0A000800385F80C3195F80C21244B1206FAD414
:10F0B000254AFF21117093F80C2142F0400283F899
:10F0C0000C21A3F52C331A68B8F1000F02D042F0DE
:10F0D000004201E022F000421A60184B320A02F0AE
:10F0E000FE0283F89C20C6F3074283F8B020360E58
:10F0F000164A83F8B460C4F84822102283F8082125
:10F10000012283F89420BF2283F8802093F8002105
:10F1100002F07F0283F8002193F8842042F001027C
:10F1200083F8842093F8842042F0100283F884202E
:10F1300084221A770020BDE8F08100BF002007403C
:10F14000FC90FF1F009EFF1F5680FF1F00A0FF1FA7
:10F150000D4B93F80C2102F0BF0283F80C21BF2263
:10F1600083F8802093F8842002F0FE0283F8842044
:10F1700093F8942002F0FE0283F894201A7F02F0A4
:10F180007B021A7700207047002007402DE9F341E9
:10F190000B460D788C78454903C902AE06E9030099
:10F1A000B3F80310B1F5007F03D90021D970022113
:10F1B0001971062D19D8AF00012CF9B201D1023115
:10F1C000C9B249083A484FF0120C0CFB01FC00EBA5
:10F1D0000C014FF6FF76B1F80080B045064604D129
:10F1E00093F80180B8F1030F01D995205BE0012C61
:10F1F000FBD891F80F80B8F1FF0F04BF4FF0000863
:10F2000081F80F80B3F8038020F80C808A73CA7BE2
:10F21000D6F84802C1F8020002F0010247EA4407AA
:10F220001743FFB2CF735A784A74D6F844220C744D
:10F2300002EBC70CB3F80380ACF80280CCF80400F2
:10F240004FF0080C02F837C0CF7BB3F8038087F08B
:10F25000010702EBC70CCCF80400ACF802804FF0B9
:10F26000480C02F837C0B3F803703844C6F84802B7
:10F2700034B9C97B12F8310060F07F0002F8310028
:10F2800058780C4A02AB03EB84042DB254F8083CC6
:10F2900012F82510012818BF43F001030B43DBB21D
:10F2A00002F82530002002B0BDE8F08124180100EA
:10F2B000FC90FF1FC0200740084610B51146FFF71D
:10F2C000B9FEFF281CD00F4B1222C0F3470002FBEF
:10F2D0000030D3F84432C27B13F8324004F07F048C
:10F2E00003F8324082F0010113F8312002F07F026E
:10F2F00003F831204FF0FF338372C372002010BD3A
:10F30000C42010BDFC90FF1F73B50D468DF807009B
:10F31000084611461646FFF78DFEFF2804461FD00B
:10F32000294632460DF10700FFF7C6FFC4F3470335
:10F3300012210D4C59436318D4F848221888121A28
:10F34000C4F848222DB2094A002002F825004FF0E7
:10F35000FF3262545A709A70DA701A715A7100E072
:10F36000962002B070BD00BFFC90FF1FC020074078
:10F370002DE9F04180460E46084611461746FFF734
:10F3800059FE0C4CC0F34700122303FB0040C57B21
:10F39000FF2D0DD03A4640463146FFF78DFF2DB286
:10F3A000D4F8443213F8352062F07B0203F835209C
:10F3B000BDE8F081FC90FF1F10B5084600211446FF
:10F3C000FFF738FE084B1222C0F3470002FB003063
:10F3D000D3F84432C27B03EBC2035A68136823603C
:10F3E0005368636010BD00BFFC90FF1F10B5084656
:10F3F0000C461146FFF71EFEFF281AD024B2104B10
:10F4000013F82430DBB213F00C0F12D09B0712D488
:10F410000C4BD3F8443213F83020D2090DD180F0D0
:10F420000100C0B213F83030DB090CBF002003200C
:10F4300010BD052010BD012010BD032010BD00BF70
:10F44000C0200740FC90FF1F08B5FFF7F3FD074BF6
:10F450001222C0F3470002FB0030C27BFF2A04D017
:10F46000D3F84432002103F8321008BDFC90FF1F8E
:10F470002DE9F041084600211E461746FFF7DAFD48
:10F48000244BC0F34700122505FB0035EC7BFF2C15
:10F490003CD0B5F80080D3F844121FFA88F24FF63A
:10F4A000FF739A4232D084F0010311F83330C3F372
:10F4B000C013D8B250BB4FEAC40C8EB901EB0C0399
:10F4C0003046A3F80280D5F802205A6011F8343093
:10F4D00003F0400363F0770301F83430BDE8F081B6
:10F4E0002B736B7301EB0C036E81964228BF16469B
:10F4F000C5F806705E805F6011F8343003F0400399
:10F5000063F0770301F83430BDE8F0819420BDE862
:10F51000F08100BFFC90FF1F2DE9F04107460C462B
:10F52000084611461546FFF785FD1A4BC0F3470004
:10F53000122606FB00361846F17BFF2927D022B29F
:10F54000154B84B196F811C0012D14BF182614264E
:10F55000BCF1010F18BF46F0010613F822C046EABD
:10F560000C0603F8226013F822606FF3410603F8DB
:10F570002260D0F84432002203F831203DB93846E9
:10F5800021462A462B46BDE8F041FFF771BFBDE892
:10F59000F08100BFFC90FF1FC02007402DE9F84319
:10F5A00008460F46012190469946FFF743FDFF2884
:10F5B00032D01B4AC0F34700122404FB0024D2F8C7
:10F5C0004452E67B15F83630DB0905EBC60223D141
:10F5D00039B2144B13F8211001F0020101F0FF00C1
:10F5E000D1B92188C4F806801FFA89F363818B4260
:10F5F000A8BF0B46207360735380C2F804800FB914
:10F60000C82305E015F8363003F0400363F07703B4
:10F6100005F83630BDE8F8839320BDE8F88300BFD5
:10F62000FC90FF1FC0200740034B044883F898104C
:10F6300001210A4600F0A8BB002007403C93FF1FB1
:10F64000054B0648002283F89420802283F80C2181
:10F650000121FF2200F098BB002007403C93FF1FD0
:10F6600038B51A4B93F8002102F07F0283F800218D
:10F6700093F80C2102F0DF0283F80C2193F880202C
:10F6800042F0200283F8802093F8842002F0DF0209
:10F6900083F8842093F8942002F0DF0283F894200A
:10F6A00093F8942042F0040283F8942044F62064F6
:10F6B0001D46013CA4B200F09DFE002CF9D195F846
:10F6C000943003F0FB0385F8943038BD00200740E8
:10F6D0002DE9FF47BA4CBB4D94F84022039995F8A9
:10F6E000803095F8847095F890608DF804200022A1
:10F6F00062F31721039101218DF8062002928DF803
:10F7000007208DF80C201F400DEB0102FF2304F5AC
:10F7100010708DF801308DF8053000F01DFB95F864
:10F720000C31D907F6B20FD59DF80130802B0BD1E3
:10F7300095F8003103F07F0385F8003195F80C311E
:10F7400003F0DF0385F80C317A0711D59D4B0420B7
:10F7500093F8A41093F8A02083F8800004AB42EA49
:10F76000012223F80E2D122001A9029300F056FB6E
:10F77000FB0749D5934D92480123BF2785F8803078
:10F7800085F8887095F89430002643F0020385F8D8
:10F790009430FF2185F898604FF4107285F800616D
:10F7A00001F088FD31464FF48062D4F8440201F044
:10F7B00081FDD4F8443203F50073C4F84832824B1B
:10F7C000FF221A7095F8943003F0FD0385F8943009
:10F7D00095F80C3143F0400385F80C319F2385F8F0
:10F7E0008C7085F8843095F8943003F0DF0385F849
:10F7F0009430102001A900F011FB95F8943003F02B
:10F80000DF0385F8943061E13D0740F1F4806D4BF2
:10F81000082283F880203209C6F3C001062A8DF839
:10F8200005208DF8071007D8C6F3800303EB820389
:10F8300019B10233DBB200E0FF23D4F84452D900FF
:10F8400068185A084FF0120C0CFB024442680292EE
:10F850004088ADF80D00E07B80F00100E07383F09C
:10F86000010615F83330C3F3801383F001039B01C5
:10F8700005F836309DF807309DF80590012B05EB13
:10F88000C60843D1DFF840A1B9F1000F14D19AF8AE
:10F890000090B9F1000F0FD1FF2349464A4601A855
:10F8A0008AF80030FFF708FD05F8369001A84946B0
:10F8B0004A464B46FFF7DCFD9AF80030012B04D096
:10F8C0009DF80530002B00F08A80BDF80DC0A3899B
:10F8D00060892288D4F8061063449BB29842A381C1
:10F8E00006D85FFA8CFC62450CD1A47B012C09D1AF
:10F8F0001944C31A9342D8BF9AB2A8F80220C8F894
:10F90000041053E00291ADF80D3068E0B9F1000F3A
:10F910001DD16B5CC3F383030D2B2B4B06D101214F
:10F920008DF806101278D2091A7010E01A78012AA0
:10F930000DD1FF21197001A84946FFF7BDFC05F85C
:10F94000369001A849464A464B46FFF791FD628929
:10F950004FF6FF739A4242D0BDF80D00A18923886B
:10F96000014489B29842A18101D18A4209D86AB37F
:10F97000B2FBF3F003FB102080B238BBA07B012860
:10F9800024D1521A9A42D8BF93B243B9D4F8022074
:10F99000C8F8042088F8023088F8033006E0D4F86C
:10F9A0000620A8F802301144C8F8041015F83630C3
:10F9B00003F0400363F0770305F8363014E000BF2E
:10F9C000FC90FF1F002007405680FF1FD4F8063030
:10F9D00002934FF0FF33ADF80D10A372E3729DF860
:10F9E000050001A900F01AFA3A4B93F8942002F0AE
:10F9F000DF0283F89420B80717D5364C022384F829
:10FA0000803094F8883094F88C201620134001A997
:10FA10008DF80C3000F002FABF2384F8883094F897
:10FA2000943003F0DF0384F89430F9061CD5294C98
:10FA3000202384F88030102384F88030142001A91A
:10FA400000F0ECF994F80C3143F0200384F80C3109
:10FA500094F8003143F0800384F8003194F8843046
:10FA600043F0200384F88430BA060DD5194C2023C6
:10FA700084F88030132001A900F0D0F994F8843084
:10FA800003F0DF0384F884303B061FD5FF2301A871
:10FA900010210DF102028DF8053000F05DF99DF89E
:10FAA0000230012B04D100228DF805208DF807309B
:10FAB000084C802384F88030172001A900F0AEF9AB
:10FAC00094F8943003F0DF0384F8943004B0BDE878
:10FAD000F08700BF002007400B4611461A4601F090
:10FAE000E9BB00BF30B50329039D049C1CD123B999
:10FAF000164A2A600422228026E040F209418B4205
:10FB000005D1022A4FF0000303D9012201E00123AD
:10FB10001A460F490C2000FB0313D9681B6951F8E2
:10FB2000221029609B5C0EE0072901D9CD2030BD51
:10FB3000074B03EB8102126A2A60002AF6D003EB1E
:10FB40004101B1F840302380002030BD5780FF1FB5
:10FB50002C180100012904D8034B5B5C13700020B2
:10FB60007047CD20704700BF4893FF1F01299DBFFC
:10FB7000024B00205A54CD20704700BF4893FF1F0E
:10FB800001298CBF002001207047054B1A788A425A
:10FB900004D05878431A58425841704701207047A2
:10FBA0004893FF1F00207047004870477C180100F1
:10FBB000012906D8044BC1EBC10119441160002092
:10FBC0007047CD20704700BF5B80FF1F012910B533
:10FBD0000DD8094BC1EBC101194408231068C45C5E
:10FBE000C81801330F2B00F8084CF7D101E0CD20E5
:10FBF00010BD002010BD00BF5B80FF1F012905D88C
:10FC0000034B03EB4101116000207047CD2070478A
:10FC10004A93FF1F012905D8034B03EB41011160F3
:10FC200000207047CD2070474E93FF1F01290AD84E
:10FC30000648136800EB41011B788B7013685B78F2
:10FC4000CB7000207047CD20704700BF4893FF1F46
:10FC500001290AD80648136800EB41011B788B7113
:10FC600013685B78CB7100207047CD20704700BFD0
:10FC70004893FF1F084B5A781A700023074AFF2148
:10FC800099540133072BF9D10023054A05219954D2
:10FC90000133072BF9D170475293FF1F5493FF1F75
:10FCA0005B93FF1F00BF7047013AD2B2062A38B5F6
:10FCB00005461C4609D8064B5A70FFF7DBFF28465D
:10FCC0002146BDE83840FFF7CFB9992038BD00BFC5
:10FCD0005293FF1F024B00225A70FFF739BA00BF40
:10FCE0005293FF1F37B50F4C257805B9B9B98DF878
:10FCF00002308DF800109DF81830ADF80320007820
:10FD00009DF81C208DF801306946FFF73FFA9DF8F9
:10FD100000302BB120B92378013B237000E09520FF
:10FD200003B030BD5293FF1F38B50A4B0C461D7807
:10FD300059788D421D4600D14CB900782146FFF715
:10FD4000E3FA2CB120B92B7801332B7038BD962003
:10FD500038BD00BF5293FF1F4B1E062B03D8094B23
:10FD600019444B7808E0CB0609D501F00F010629AC
:10FD700005D8044B19444B7A137000207047822039
:10FD8000704700BF5293FF1F4B1E062B2DE9F04119
:10FD90008046154603D8164B19444A7021E0CB061D
:10FDA00022D501F00F04062C1ED8012A4FEAD116E5
:10FDB0000F4F04D121463246FFF7DAFA0FE072B94D
:10FDC0003B195B7A012B0AD121463246FFF7A4FB8F
:10FDD0002CB94046214686F00102FFF79DFB3C44CA
:10FDE00065720020BDE8F0818220BDE8F08100BF8F
:10FDF0005293FF1F00207047062903D9A1F1100379
:10FE0000072B07D8044B53F82130002B14BF0020D8
:10FE1000C4207047C4207047A4180100102838B5CA
:10FE200004460D4601D1FFF725FF044B53F824305B
:10FE30000BB128469847002038BD00BFA418010028
:10FE40001FB504A9144601F8090D02221A800846BC
:10FE50000DF10F020521FFF77FFF034B9DF80F20E7
:10FE60001A80236004B010BD6493FF1F1FB504A95E
:10FE7000144601F8090D01221A8008460DF10F02FF
:10FE80000421FFF769FF044B9DF80F201A80002022
:10FE9000236004B010BD00BF6493FF1F7FB5002432
:10FEA0001C8049888DF80700ADF80E10FFF768FE3A
:10FEB00000B3BDF80E20114E131B5A425A410DF1EA
:10FEC00007000121FFF760FF9DF80E200DF10700EC
:10FED0000421FFF759FF73680DF10E020546012159
:10FEE0009DF80700984773689DF807000221224695
:10FEF000984700E00425284604B070BD6493FF1FB6
:10FF000037B502AA002402F8010D0D461C801046E8
:10FF100001210422FFF738FF6A88024B20461A723B
:10FF200003B030BD6493FF1F37B54C888D888DE8D2
:10FF30000C00210AE2B22B46FFF7D4FD03B030BD1E
:10FF40002DE9F04186B00F461E4600238DF80F00C4
:10FF50000593904603230DF10F00012104AA8DF8AB
:10FF60001030FFF7F9FE3D78274C15F0030525D139
:10FF700006210DF111020DF10F00FFF7EDFE9DF8C6
:10FF800011309DF80F0003F00303238005AB0093AD
:10FF90000DF11203019302212B462A46FFF7A2FD21
:10FFA000059BDB7913F0400F238814BF43F0010356
:10FFB00023F001032380022333801FE0012D09D1A8
:10FFC0009DF81020BB88012A02D113F0FF0F14D135
:10FFD0000023EFE7022D11D1397941F010010DF125
:10FFE0000F00C9B20DF11202FFF7B6FE9DF81230F4
:10FFF00003F001032380358000E0CD20C8F80040E5
:020000021000EC
:1000000006B0BDE8F08100BF6493FF1F7FB50022FA
:100010001A800B784E788DF8070013F003030D4615
:10002000C6F3400632D1B6B14B88013B9BB2012BDF
:1000300050D80DF1070006210DF10F02FFF78CFEDD
:100040000446002847D1AA789DF80F3006FA02F23C
:100050001A43D2B211E04E88012E3BD10DF10700B8
:1000600006210DF10F02FFF777FE044698BBAA7830
:100070009DF80F30964023EA06020DF10700062195
:100080008DF80F20FFF780FE044624E0022B21D1DB
:1000900009798DF80F100DF1070041F0100132467B
:1000A000FFF772FE6B78002E0CBF08210721012B91
:1000B000044607D19DF80F1001F00F00C909FFF7A2
:1000C000C3F90821054B9DF807005B680DF10F028D
:1000D000984700E0CD24204604B070BD6493FF1F14
:1000E00010B500241C800B7803F00303012B0A4693
:1000F00005D109799278FFF739FD204610BD04201B
:1001000010BD38B50C7804F00304012C154607D156
:100110001C80044C09792246FFF71CFD2C6038BD79
:10012000042038BD6493FF1F13B5CD298DF8070057
:1001300006D10DF1070090210122FFF725FE18E0FE
:100140000D481C88018A12688C4288BF19800446B9
:100150001B889DF807000021FEF756FF94F90A302E
:10016000002B06DA00210DF107000A460B46FFF7C7
:100170007FF902B010BD00BF6493FF1F73B5054641
:1001800000266A4601218DF800600196FFF7E4FD24
:10019000AA783F4C012A46D168680368C4F80A303F
:1001A0004368A07AC4F80E3004F10A0110F0600F21
:1001B000238A13D1E37A374850F82340002C5ED0CD
:1001C0009DF80020022A5AD803EB43031844024446
:1001D00092F83430012B52D1287818E0202BADF85A
:1001E00002301AD873B102060CD40A68C4F812207F
:1001F0004A68C4F816202846314604F11A02FFF76F
:1002000037F943E0E46B002C39D02878224901AA61
:100210000DF10203A047014632E002A82B7800F856
:10022000073D902113E09DF80030042B12D12B786C
:10023000217A02AD05F8063D2846FFF7F5F90121C0
:100240000A462846FFF7A0FD227A28460321FFF739
:100250009BFD1BE094F90A30002B17DBEB78ABB960
:10026000E66B66B1B5F8093028780833ADF802308E
:1002700004F1120101AA0DF10203B047CBE7CD2131
:10028000287801AA0DF10203FFF74EFF02B070BDFE
:100290006493FF1F041901006E93FF1F034B596005
:1002A000DA630021024AFFF7A5BD00BF6493FF1F78
:1002B0007D01010007B502AB054A03F8010D0021DD
:1002C00018465160D163FFF797FD03B05DF804FB5A
:1002D0006493FF1F00207047354B41F24802995844
:1002E00021F00F0141F00201995041F204029958A6
:1002F00041F48021995041F23402995841F480210F
:10030000995003F52C33602193F8942042F00202B7
:1003100083F89420C02283F80021FF221A7483F806
:10032000802083F8882083F88420002283F88C20A2
:1003300083F80C111F491A75080A00F0FE0083F8B3
:10034000982083F8C02083F8C42083F8C82083F85D
:10035000CC2083F8D02083F8D42083F8D82083F8E9
:10036000DC2083F8E02083F8E42083F8E82083F899
:10037000EC2083F8F02083F8F42083F8F82083F849
:10038000FC2083F89C00C1F30740090E83F8B000FD
:1003900083F8B41083F8AC201A7783F8082193F817
:1003A000942002F0D40242F0010283F894207047B6
:1003B00000700440009EFF1F024B4FF400125A6071
:1003C000704700BF00E100E0034B4FF40012C3F898
:1003D00084215A60704700BF00E100E010B5FEF7CD
:1003E0008DF9044618B9FFF7EFFF204610BD1B201A
:1003F00010BD00BF034B4AF202629A814BF2804269
:100400009A8170470020054081F0004102E000BF62
:1004100083F0004330B54FEA41044FEA430594EAC4
:10042000050F08BF90EA020F1FBF54EA000C55EAFF
:10043000020C7FEA645C7FEA655C00F0E2804FEAD0
:100440005454D4EB5555B8BF6D420CDD2C4480EAB2
:10045000020281EA030382EA000083EA010180EAE2
:10046000020281EA0303362D88BF30BD11F0004F30
:100470004FEA01314FF4801C4CEA113102D0404266
:1004800061EB410113F0004F4FEA03334CEA1333A1
:1004900002D0524263EB430394EA050F00F0A780B9
:1004A000A4F10104D5F1200E0DDB02FA0EFC22FAB4
:1004B00005F2801841F1000103FA0EF2801843FAA8
:1004C00005F359410EE0A5F120050EF1200E012A99
:1004D00003FA0EFC28BF4CF0020C43FA05F3C018D7
:1004E00051EBE37101F0004507D54FF0000EDCF150
:1004F000000C7EEB00006EEB0101B1F5801F1BD3F9
:10050000B1F5001F0CD349085FEA30004FEA3C0CFC
:1005100004F101044FEA445212F5800F80F09A80F2
:10052000BCF1004F08BF5FEA500C50F1000041EBF6
:10053000045141EA050130BD5FEA4C0C404141EBFA
:10054000010111F4801FA4F10104E9D191F0000F21
:1005500004BF01460020B1FA81F308BF2033A3F1A4
:100560000B03B3F120020CDA0C3208DD02F1140C9B
:10057000C2F10C0201FA0CF021FA02F10CE002F1D6
:100580001402D8BFC2F1200C01FA02F120FA0CFCCF
:10059000DCBF41EA0C019040E41AA2BF01EB045118
:1005A000294330BD6FEA04041F3C1CDA0C340EDC16
:1005B00004F11404C4F1200220FA04F001FA02F359
:1005C00040EA030021FA04F345EA030130BDC4F117
:1005D0000C04C4F1200220FA02F001FA04F340EA0C
:1005E0000300294630BD21FA04F0294630BD94F0BD
:1005F000000F83F4801306BF81F480110134013DA4
:100600004EE77FEA645C18BF7FEA655C29D094EA14
:10061000050F08BF90EA020F05D054EA000C04BF92
:100620001946104630BD91EA030F1EBF002100207D
:1006300030BD5FEA545C05D14000494128BF41F01C
:10064000004130BD14F580043CBF01F5801130BD80
:1006500001F0004545F0FE4141F470014FF000000B
:1006600030BD7FEA645C1ABF194610467FEA655CBC
:100670001CBF0B46024650EA013406BF52EA03355E
:1006800091EA030F41F4002130BD00BF90F0000F4C
:1006900004BF0021704730B54FF4806404F1320488
:1006A0004FF000054FF0000150E700BF90F0000F41
:1006B00004BF0021704730B54FF4806404F1320468
:1006C00010F0004548BF40424FF000013EE700BF38
:1006D00042004FEAE2014FEA31014FEA02701FBFC8
:1006E00012F07F4393F07F4F81F06051704792F09A
:1006F000000F14BF93F07F4F704730B54FF4607414
:1007000001F0004521F0004120E700BF50EA01025E
:1007100008BF704730B54FF000050AE050EA01020B
:1007200008BF704730B511F0004502D5404261EB7B
:1007300041014FF4806404F132045FEA915C3FF4BC
:10074000DCAE4FF003025FEADC0C18BF03325FEA55
:10075000DC0C18BF033202EBDC02C2F1200300FA0A
:1007600003FC20FA02F001FA03FE40EA0E0021FA2F
:1007700002F11444C1E600BF70B54FF0FF0C4CF419
:10078000E06C1CEA11541DBF1CEA135594EA0C0FCF
:1007900095EA0C0F00F0DEF82C4481EA030621EA0A
:1007A0004C5123EA4C5350EA013518BF52EA033545
:1007B00041F4801143F4801338D0A0FB02CE4FF0F7
:1007C0000005E1FB02E506F00042E0FB03E54FF027
:1007D0000006E1FB03569CF0000F18BF4EF0010E1F
:1007E000A4F1FF04B6F5007F64F5407404D25FEA1B
:1007F0004E0E6D4146EB060642EAC62141EA5551CE
:100800004FEAC52040EA5E504FEACE2EB4F1FD0C0F
:1008100088BFBCF5E06F1ED8BEF1004F08BF5FEA8D
:10082000500E50F1000041EB045170BD06F000463F
:1008300046EA010140EA020081EA0301B4EB5C04EC
:10084000C2BFD4EB0C0541EA045170BD41F48011E4
:100850004FF0000E013C00F3AB8014F1360FDEBF09
:10086000002001F0004170BDC4F10004203C35DAE5
:100870000C341BDC04F11404C4F1200500FA05F368
:1008800020FA04F001FA05F240EA020001F0004209
:1008900021F0004110EBD37021FA04F642EB06017F
:1008A0005EEA430E08BF20EAD37070BDC4F10C04A9
:1008B000C4F1200500FA04F320FA05F001FA04F26D
:1008C00040EA020001F0004110EBD37041F1000159
:1008D0005EEA430E08BF20EAD37070BDC4F1200564
:1008E00000FA05F24EEA020E20FA04F301FA05F2CC
:1008F00043EA020321FA04F001F0004121FA04F274
:1009000020EA020000EBD3705EEA430E08BF20EA43
:10091000D37070BD94F0000F0FD101F0004640007D
:1009200041EB010111F4801F08BF013CF7D041EAFF
:10093000060195F0000F18BF704703F00046520003
:1009400043EB030313F4801F08BF013DF7D043EAD4
:100950000603704794EA0C0F0CEA135518BF95EA8A
:100960000C0F0CD050EA410618BF52EA4306D1D111
:1009700081EA030101F000414FF0000070BD50EA30
:10098000410606BF1046194652EA430619D094EABA
:100990000C0F02D150EA013613D195EA0C0F05D1A4
:1009A00052EA03361CBF104619460AD181EA0301F8
:1009B00001F0004141F0FE4141F470014FF00000B0
:1009C00070BD41F0FE4141F4780170BD70B54FF04B
:1009D000FF0C4CF4E06C1CEA11541DBF1CEA1355CB
:1009E00094EA0C0F95EA0C0F00F0A7F8A4EB0504AD
:1009F00081EA030E52EA03354FEA013100F08880A4
:100A00004FEA03334FF0805545EA131343EA12636C
:100A10004FEA022245EA111545EA10654FEA002621
:100A20000EF000419D4208BF964244F1FD0404F5DA
:100A3000407402D25B084FEA3202B61A65EB030536
:100A40005B084FEA32024FF480104FF4002CB6EBF3
:100A5000020E75EB030E22BFB61A754640EA0C0073
:100A60005B084FEA3202B6EB020E75EB030E22BFB3
:100A7000B61A754640EA5C005B084FEA3202B6EBF4
:100A8000020E75EB030E22BFB61A754640EA9C00B3
:100A90005B084FEA3202B6EB020E75EB030E22BF83
:100AA000B61A754640EADC0055EA060E18D04FEA41
:100AB000051545EA16754FEA06164FEAC30343EAE1
:100AC00052734FEAC2025FEA1C1CC0D111F4801FAE
:100AD0000BD141EA00014FF000004FF0004CB6E7A7
:100AE00011F4801F04BF01430020B4F1FD0C88BF46
:100AF000BCF5E06F3FF6AFAEB5EB030C04BFB6EB51
:100B0000020C5FEA500C50F1000041EB045170BD43
:100B10000EF0004E4EEA113114EB5C04C2BFD4EB70
:100B20000C0541EA045170BD41F480114FF0000EF4
:100B3000013C90E645EA060E8DE60CEA135594EA70
:100B40000C0F08BF95EA0C0F3FF43BAF94EA0C0F73
:100B50000AD150EA01347FF434AF95EA0C0F7FF4E8
:100B600025AF104619462CE795EA0C0F06D152EA3C
:100B700003353FF4FDAE1046194622E750EA410620
:100B800018BF52EA43067FF4C5AE50EA41047FF431
:100B90000DAF52EA43057FF4EBAE12E74FF0FF3C96
:100BA00006E000BF4FF0010C02E000BF4FF0010C67
:100BB0004DF804CD4FEA410C7FEA6C5C4FEA430CE0
:100BC00018BF7FEA6C5C1BD001B050EA410C0CBF2F
:100BD00052EA430C91EA030F02BF90EA020F002091
:100BE000704710F1000F91EA030F58BF994208BFF8
:100BF00090422CBFD8176FEAE37040F001007047B5
:100C00004FEA410C7FEA6C5C02D150EA013C07D10B
:100C10004FEA430C7FEA6C5CD6D152EA033CD3D056
:100C20005DF8040B704700BF8446104662468C4650
:100C30001946634600E000BF01B5FFF7B7FF002883
:100C400048BF10F1000F01BD4DF808EDFFF7F4FFAC
:100C50000CBF012000205DF808FB00BF4DF808ED37
:100C6000FFF7EAFF34BF012000205DF808FB00BF5A
:100C70004DF808EDFFF7E0FF94BF012000205DF87C
:100C800008FB00BF4DF808EDFFF7CEFF94BF012031
:100C900000205DF808FB00BF4DF808EDFFF7C4FF2A
:100CA00034BF012000205DF808FB00BF4FEA41027D
:100CB00012F5001215D211D56FF47873B3EB6252AE
:100CC00012D94FEAC12343F0004343EA505311F0D5
:100CD000004F23FA02F018BF404270474FF0000067
:100CE000704750EA013005D111F0004008BF6FF0A5
:100CF000004070474FF00000704700BF80F0004098
:100D000002E000BF81F0004142001FBF5FEA4103E3
:100D100092EA030F7FEA226C7FEA236C6AD04FEAE3
:100D20001262D2EB1363C1BFD21841404840414028
:100D3000B8BF5B42192B88BF704710F0004F40F4DA
:100D4000000020F07F4018BF404211F0004F41F4F6
:100D5000000121F07F4118BF494292EA030F3FD0C2
:100D6000A2F1010241FA03FC10EB0C00C3F12003D5
:100D700001FA03F100F0004302D5494260EB400064
:100D8000B0F5000F13D3B0F1807F06D340084FEACF
:100D9000310102F10102FE2A51D2B1F1004F40EBC4
:100DA000C25008BF20F0010040EA0300704749002C
:100DB00040EB000010F4000FA2F10102EDD1B0FAF7
:100DC00080FCACF1080CB2EB0C0200FA0CF0AABFEC
:100DD00000EBC25052421843BCBFD040184370478A
:100DE00092F0000F81F4000106BF80F40000013290
:100DF000013BB5E74FEA41037FEA226C18BF7FEA67
:100E0000236C21D092EA030F04D092F0000F08BFA8
:100E10000846704790EA010F1CBF0020704712F08F
:100E20007F4F04D1400028BF40F00040704712F1CE
:100E300000723CBF00F50000704700F0004343F033
:100E4000FE4040F4000070477FEA226216BF084669
:100E50007FEA23630146420206BF5FEA412390EA2C
:100E6000010F40F4800070474FF0000304E000BF22
:100E700010F0004348BF40425FEA000C08BF7047D3
:100E800043F0964301464FF000001CE050EA010297
:100E900008BF70474FF000030AE000BF50EA0102AC
:100EA00008BF704711F0004302D5404261EB410199
:100EB0005FEA010C02BF84460146002043F0B643BE
:100EC00008BFA3F18053A3F50003BCFA8CF2083AE3
:100ED000A3EBC25310DB01FA02FC634400FA02FCEC
:100EE000C2F12002BCF1004F20FA02F243EB0200F3
:100EF00008BF20F00100704702F1200201FA02FC55
:100F0000C2F1200250EA4C0021FA02F243EB020047
:100F100008BF20EADC7070474FF0FF0C1CEAD0528B
:100F20001EBF1CEAD15392EA0C0F93EA0C0F6FD04C
:100F30001A4480EA010C400218BF5FEA41211ED02A
:100F40004FF0006343EA501043EA5111A0FB013116
:100F50000CF00040B1F5000F3EBF490041EAD371EB
:100F60005B0040EA010062F17F02FD2A1DD8B3F167
:100F7000004F40EBC25008BF20F00100704790F0D6
:100F8000000F0CF0004C08BF49024CEA502040EA28
:100F900051207F3AC2BFD2F1FF0340EAC2507047EE
:100FA00040F400004FF00003013A5DDC12F1190F2C
:100FB000DCBF00F000407047C2F10002410021FA9E
:100FC00002F1C2F1200200FA02FC5FEA310040F1B6
:100FD000000053EA4C0308BF20EADC70704792F02F
:100FE000000F00F0004C02BF400010F4000F013A67
:100FF000F9D040EA0C0093F0000F01F0004C02BF62
:10100000490011F4000F013BF9D041EA0C018FE7D0
:101010000CEAD15392EA0C0F18BF93EA0C0F0AD0D6
:1010200030F0004C18BF31F0004CD8D180EA0100FC
:1010300000F00040704790F0000F17BF90F0004F95
:10104000084691F0000F91F0004F14D092EA0C0F77
:1010500001D142020FD193EA0C0F03D14B0218BF0A
:10106000084608D180EA010000F0004040F0FE4050
:1010700040F40000704740F0FE4040F440007047EC
:101080004FF0FF0C1CEAD0521EBF1CEAD15392EA6B
:101090000C0F93EA0C0F69D0A2EB030280EA010C5B
:1010A00049024FEA402037D04FF0805343EA1111F4
:1010B00043EA10130CF000408B4238BF5B0042F152
:1010C0007D024FF4000C8B4224BF5B1A40EA0C00F7
:1010D000B3EB510F24BFA3EB510340EA5C00B3EB29
:1010E000910F24BFA3EB910340EA9C00B3EBD10F17
:1010F00024BFA3EBD10340EADC001B0118BF5FEA69
:101100001C1CE0D1FD2A3FF650AF8B4240EBC25091
:1011100008BF20F0010070470CF0004C4CEA502052
:101120007F32C2BFD2F1FF0340EAC250704740F4A1
:1011300000004FF00003013A37E792F0000F00F093
:10114000004C02BF400010F4000F013AF9D040EA11
:101150000C0093F0000F01F0004C02BF490011F4A5
:10116000000F013BF9D041EA0C0195E70CEAD1539D
:1011700092EA0C0F08D142027FF47DAF93EA0C0F84
:101180007FF470AF084676E793EA0C0F04D14B0268
:101190003FF44CAF08466EE730F0004C18BF31F01A
:1011A000004CCAD130F000427FF45CAF31F0004314
:1011B0007FF43CAF5FE700BFFDF737F9002100F097
:1011C00004B80C4B5B58435004310B480B4B42188E
:1011D0009A42FFF4F6AF0A4A00F003B80023136006
:1011E0000432084B9A42FFF4F9AF00F00DF8804743
:1011F00070470000981901000880FF1F6885FF1FD5
:101200000086FF1F00A2FF1F274C08B5F7F72DF936
:10121000F7F790F9F7F7DAFAF7F7EEFAF7F7F2F9E6
:10122000F7F7ACFCFCF7FEF8FBF7CAFEF7F717FE82
:10123000F7F770FBE08CF7F763FC2078F7F7F2F92B
:10124000E078F7F75FFAF7F70DFC28B1F7F70AFC3B
:101250006070F7F707FCA060F7F76CFC60792189F4
:10126000228AFBF707FFFCF76EFEFCF7F9FF0F4B36
:101270004FF400725A60FAF707FCFBF7D3F80C4BF7
:1012800004225A60FAF724FDFBF7F0F8FBF7CBF8DD
:10129000F7F7F0FBF7F724FC0028F3D0FCF753FE38
:1012A000FAF7F2FBEEE700BF0C80FF1F80F00F4063
:1012B00000F00F40F0B4840743D0541E002A3ED003
:1012C000CDB2034603E0621E002C38D0144603F86A
:1012D000015B9A07F7D1032C2AD9CDB245EA05253F
:1012E0000F2C45EA054515D9A4F110073F0903F174
:1012F000100606EB07161A46156055609560D56016
:101300001032B242F8D104F00F040137032C03EB82
:1013100007130DD91E462246043A032A46F8045BF9
:10132000FAD8221F22F003020432134404F003040B
:101330002CB1C9B21C4403F8011BA342FBD1F0BC81
:10134000704714460346C6E7C1F30A5CF8B5ACF231
:10135000FF33132B06460F4610DC002B39DBDFF87A
:1013600088C04CFA03F303EA010C5CEA000C1AD1C2
:1013700007F000416046C2E90067F8BD332B1CDC72
:101380004FF0FF33ACF2134C23FA0CFC1CEA0003C1
:1013900019D020EA0C060F46C2E900670B46324618
:1013A000FFF736F8F8BD21EA03070026C2E9006717
:1013B0003B463246FFF72CF8F8BD07F0004100200D
:1013C000C2E90067F8BD07F000411846C2E90067AE
:1013D000F8BD07F00041002004460D46304639466E
:1013E000C2E90045F8BD00BFFFFF0F00024B13B17B
:1013F000024800F005B87047000000000D1401001D
:10140000014600200246034600F018B838B5094DE1
:10141000094C641BA41018BF05EB840505D0013CE2
:1014200055F8043D9847002CF9D1BDE8384000F04C
:10143000A7BA00BF9419010098190100F0B5274C14
:101440002668D6F8484185B00746002C41D065682B
:101450001F2D1EDD224818B94FF0FF3005B0F0BD3A
:101460004FF4C870039102920193AFF30080039987
:10147000029A019B04460028EED0D6F84851256018
:10148000002060600546C6F84841C4F88801C4F8E9
:101490008C013FB9AB1C00200135656044F8231076
:1014A00005B0F0BD04EB85004FF0010CC0F88820BA
:1014B000D4F888610CFA05F21643022FC4F888614B
:1014C000C0F80831E6D1D4F88C311A43C4F88C2125
:1014D000E0E706F5A674C6F84841B8E770190100C0
:1014E00000000000000000002DE9F84FC1F30A578A
:1014F000A7F2FF36132E02460B4604460D468946D8
:101500008A46804622DC002E54DB3D4F374107EAF5
:10151000010C5CEA000C1ED037A3D3E90023FEF7D0
:1015200079FF00220023FFF7B7FB58B1002D05DD3E
:101530004FF4801A4AFA06F606EB050A2AEA07096A
:101540004FF0000840464946BDE8F88F332E06DDCF
:10155000B6F5806F43D010461946BDE8F88FA7F264
:10156000134C4FF0FF3B2BFA0CFB1BEA000FF2D0A1
:1015700021A3D3E90023FEF74DFF00220023FFF74C
:101580008BFB0028DED0002D0DDD142E09D0C7F511
:10159000866703374FF0010808FA07F818EB0408CC
:1015A00001D305F1010A28EA0B08D1464046494615
:1015B000BDE8F88F10A3D3E90023FEF72BFF00222C
:1015C0000023FFF769FB0028BCD0002D0DDB55EA96
:1015D000040808D0DFF82C904FF00008B2E7FEF7BF
:1015E00019FFBDE8F88FC146ACE74FF000084FF097
:1015F0000049A7E7AFF300809C7500883CE4377E84
:10160000FFFF0F000000F03F2DE9F84FC1F30A572C
:10161000A7F2FF36132E02460B4604460D468946B6
:101620008A4680461CDC002E40DB3D4F374107EAEE
:10163000010C5CEA000C18D037A3D3E90023FEF7B5
:10164000E9FE00220023FFF727FB28B1002D42DB33
:101650002AEA07094FF0000840464946BDE8F88FDE
:10166000332E06DDB6F5806F31D010461946BDE841
:10167000F88FA7F2134C4FF0FF3B2BFA0CFB1BEA41
:10168000000FF2D024A3D3E90023FEF7C3FE00220B
:101690000023FFF701FB0028DED0002D22DB28EA23
:1016A0000B08D14640464946BDE8F88F1AA3D3E956
:1016B0000023FEF7AFFE00220023FFF7EDFA00281B
:1016C000CAD0002D1CDB4FF00008C146C4E7FEF76E
:1016D000A1FEBDE8F88F4FF4801A4AFA06F606EB31
:1016E000050AB5E7142E14D0C7F586670123033722
:1016F00003FA07F717EB040828BF05EB030ACEE748
:1017000025F00042074B224318BF99464FF00008CE
:10171000A2E705F1010AC2E79C7500883CE4377E28
:10172000FFFF0F000000F0BF8025000040380000E0
:10173000004B0000807000000096000000E10000F7
:10174000002C010000C201000084030090D00300BF
:1017500020A1070040420F0050C300008813000082
:10176000018008080000000000000000C800000020
:101770000100C80000800000000000000000000020
:101780000000000000000000000000000000000059
:10179000000000000000000001000200040008003A
:1017A0001000200001010100010000000000000005
:1017B0000000000000010000000000000001000027
:1017C0000000000001010100000000000000000016
:1017D0000001000000000000010101000101000102
:1017E00001000000010101000000000000000000F5
:1017F00000010000000000000101010001010001E2
:1018000001000000000000000000000000000101D5
:1018100001000001000000000000000000000101C4
:101820000100000108000000040000005780FF1FB5
:10183000040000000904000090180100A018010035
:101840000000000000000000000000000000000098
:101850002E81FF1FEB80FF1F000000000000000032
:101860000000000000000000000000000000120066
:10187000430000000000000000000000030102011E
:10188000100002020010000303011000000100001C
:101890005780FF1FB180FF1F8B80FF1F6980FF1FD4
:1018A000043A26227D01010081EA000015EB0000C8
:1018B00085E80000A5FC0000A5FC0000A5FC0000D8
:1018C000A5FC0000A5FC0000A5FC0000A5FC000094
:1018D000A5FC0000A5FC0000A5FC0000A5FC000084
:1018E000A5FC000017EE0000B1ED00000DEE0000B9
:1018F000D9ED0000B1ED0000A5FC000099ED00005D
:1019000085EE000041FF00000D0001000000000016
:101910000D0001000000000001FF000029FF000091
:10192000000000006DFE00009DFE000003010100AC
:10193000E100010041FE0000010100010100000082
:101940000001010000000000010101010100000090
:101950000101000101000100000100000100000080
:10196000363231305631303500000000430000007F
:101970004081FF1FF8B500BFF8BC08BC9E46704709
:0C198000F8B500BFF8BC08BC9E467047DC
:08198C00ED1301003584000099
:0419940011840000BA
:1019980060190100000102000008000001000000B9
:1019A800020000000000000000000000000000002D
:1019B800000000000000000000000000000000001F
:1019C800000000000000000000000000000000000F
:1019D80000000000A1200000000002000000FF0439
:1019E80003090400C2010000000800000000000014
:1019F80000220342004100440020005300540052DA
:101A08000049004E004700200049004E00440045B0
:101A180000580026035300740065007000700065CC
:101A280000720020004D006F0074006F00720020EB
:101A38000044006500760020003A03540052004933
:101A4800004E0041004D004900430020004D006F4A
:101A580000740069006F006E00200043006F006E84
:101A680000740072006F006C00200020002000202D
:101A780000200009024300020100C03209040000EE
:101A880001020200000524001001052401010104DF
:101A980024020605240600010705830310000A092D
:101AA800040100020A000000070581021000000777
:101AB80005020210000012010002020000103C2A78
:101AC8000001020001020001000000002C84FF1F39
:101AD8009484FF1FFC84FF1F00000000000000002A
:101AE80000000000000000000000000000000000EE
:101AF8000000000000000000000000006C19010058
:101B080000000000000000000000000000000000CD
:101B180000000000000000000000000000000000BD
:101B280000000000000000000000000000000000AD
:101B3800000000000000000000000000000000009D
:101B4800000000000000000000000000000000008D
:101B5800000000000000000000000000000000007D
:101B6800000000000000000000000000000000006D
:101B780001000000000000000E33CDAB34126DE60A
:101B8800ECDE05000B000000000000000000000073
:101B9800000000000000000000000000000000003D
:101BA800000000000000000000000000000000002D
:101BB800000000000000000000000000000000001D
:101BC800000000000000000000000000000000000D
:101EF800981901000880FF1F60050000000000001D
:081F08000000000000000000D1
:020000020000FC
:020000041FFFDC
:04800000000000007C
:04000003100011B91F
:00000001FF
